:020000040800F2
:1000000000000220F92000083F21000841210008DB
:100010004321000845210008472100080000000096
:10002000000000000000000000000000492100085E
:100030004B210008000000004D2100084F2100085E
:1000400053210008552100085721000859210008B4
:100050005B2100085D2100082926000841260008D0
:100060005926000871260008892600086921000821
:100070006B2100086D2100086F2100087121000824
:1000800073210008752100087721000879210008F4
:100090007B2100087D2100087F210008A12600089F
:1000A0008321000885210008872100088921000894
:1000B0008B210008D91C00088F210008912100081D
:1000C0009321000895210008972100089921000834
:1000D0009B2100089D2100089F210008A121000804
:1000E00005270008A5210008A7210008A92100086C
:1000F000AB210008AD210008AF210008B1210008A4
:10010000B3210008B5210008091B0008B921000827
:10011000BB210008BD210008BF210008C121000843
:10012000111C0008C5210008C7210008C9210008CA
:10013000CB210008CD210008CF210008D1210008E3
:10014000D3210008D5210008D7210008D9210008B3
:10015000DB210008DD210008DF210008E121000883
:10016000E3210008E5210008E7210008E921000853
:10017000EB210008ED210008EF210008F121000823
:10018000F3210008F521000810B5054C237833B998
:10019000044B13B10448AFF300800123237010BD5A
:1001A0000402002000000000D4B10008084B10B584
:1001B0001BB108490848AFF300800848036803B939
:1001C00010BD074B002BFBD0BDE81040184700BF07
:1001D0000000000008020020D4B100080402002042
:1001E00000000000162031A1ABBE30484168002954
:1001F00001D0364A11600168002901D132490160FD
:100200008168C268002900D08D46002A01D002F51D
:10021000807A00218B460F462548264A121A07F09D
:10022000CBFC06F0F9FF152025A1ABBE2449002028
:1002300001B40B780131002B15D0202BF9D0222BE3
:1002400001D0272B01D11A0001E02022013902B48C
:1002500001300B780131002B05D09A42F9D10022F0
:100260004B1E1A70E5E76946020092006A446B462D
:100270009A4206D9043A14681D6815601C6004335C
:10028000F6E76C460725AC43A54604000D000A4876
:10029000002802D00948AFF3008007F067FC200077
:1002A000290001F041FC07F04DFC00BF00000020D8
:1002B00004020020385F0020000000000000000061
:1002C00010000020FF000000385F00209401002093
:1002D000C3785BB9037818485A09203203F01F032A
:1002E000012101FA03F340F822307047F0B4134BB8
:1002F0004778D968827804780F4EC943C1F3022148
:10030000C1F10405EDB20F2307FA05F50B41EDB27B
:1003100013402B4304F1604202F561421B01DBB242
:1003200082F800330378012203F01F015B098A4041
:1003300046F82320F0BC704700E100E000ED00E04B
:10034000F0B444680A680D790F4B24F0407424F42B
:100350008074224342EA0522426001F1080294CAF5
:1003600086684D793C4322433340134343EA4503B7
:1003700083600A7DC36A013AD2B223F4700343EA70
:100380000253C362F0BC7047FDF7FFC070B4074D65
:10039000066842688468C168054B68683243224336
:1003A0000A43034013436B6070BC70470023014055
:1003B000E030FCFF836819B923F0010383607047C4
:1003C00043F0010383607047092970B41DD9A1F17E
:1003D0000A0606EB4606C5680724B440B34025EA82
:1003E00004042343062AC3601BD90C2A27D90D3ADB
:1003F00002EB8202C36A1F24944001FA02F223EA4C
:1004000004010A43C26270BC704701EB41060569F2
:100410000724B440B34025EA04042343062A0361B9
:10042000E3D8013A02EB8202436B1F24944001FAA5
:1004300002F223EA04010A43426370BC7047073AA0
:1004400002EB8202036B1F24944001FA02F223EABA
:1004500004010A43026370BC704700BF836819B986
:1004600023F480738360704743F480738360704724
:10047000836819B923F400738360704743F40073F1
:1004800083607047F0B40F684E68094D8C68CA6885
:100490002B6847EA06010C4340F6FE712243814077
:1004A00023EA010302FA00F003432B60F0BC70471B
:1004B0000074004041B9084901220B6802FA00F0BB
:1004C00023EA000008607047034901220B6802FA22
:1004D00000F01843086070470074004049B90949AA
:1004E0004FF480520B6802FA00F023EA0000086023
:1004F000704704494FF480520B6802FA00F0184329
:10050000086070470074004002683749002310B447
:1005100022F001022124884202600360436083606C
:10052000C360036144614DD0304B984235D0304BAD
:10053000984239D02F4B98423DD02F4B984247D00C
:100540002E4B984248D02E4B98421DD02D4B9842AE
:100550001ED02D4B984243D02C4B98421DD02C4B93
:10056000984221D02B4B984225D02B4B98422FD02C
:100570002A4B984230D02A4B984205D0294B9842BA
:1005800006D05DF8044B7047274A43F8942CF8E7EF
:100590004FF03D5243F8AC2CF3E74FF4746243F84C
:1005A000202C5DF8044B70474FF4741243F8382C3C
:1005B0005DF8044B70474FF0746243F8502C5DF8BF
:1005C000044B7047194B3D229A605DF8044B70470D
:1005D000174A43F8642CD4E7164A43F87C2CD0E73A
:1005E0003D2243F8082CCCE710600240286002400E
:1005F00040600240586002407060024088600240E3
:10060000A0600240B86002401064024028640240CA
:1006100040640240586402407064024088640240B2
:10062000A0640240B864024000003D200060024027
:100630003D000020400F0020F0B401F118028CCAE8
:100640000E68CD684C693543254315434E6A4C6BA3
:100650008A6B1D433D438B6A35431D4306680B4B34
:100660002C432243334013430360CC6A42690B6B33
:1006700022F007022343134343610B6943604B6835
:1006800083608B68C360F0BC704700BF3F801CF084
:10069000036819B923F001030360704743F00103B5
:1006A00003607047036822B923F4002303600161EB
:1006B000704743F40023036001617047036819B970
:1006C00023F480230360704743F480230360704762
:1006D00010B4094B094C0A4AA04294BF1846104670
:1006E00011F0005F21F0F02121F0821114BFC160F0
:1006F00081605DF8044B7047006002400F64024067
:10070000006402400B060CD54369AAB143F0800394
:10071000802943610FD0036801F01E011943016075
:100720007047802907D0002AF5D1036801F01E0127
:1007300023EA01010160704723F0800380294361AF
:10074000F3D170470022F0B513460126032704E0D9
:100750000133102B02F102022FD00D6806FA03F4C8
:1007600034EA0505F4D1D0F800E007FA02F5ED43CC
:100770000EEA050EC0F800E091F804E0D0F800C0E1
:100780000EFA02FE4EEA0C0EC0F800E091F804E00A
:100790000EF1FF3EBEF1010F07FA02FC0ED9C4684C
:1007A00024EA0C04C460CC79C568944001332C431E
:1007B000102BC46002F10202CFD1F0BDD0F808E0E6
:1007C00005EA0E05856091F805E085680EFA02FEDF
:1007D0004EEA05058560456825EA040444608C7985
:1007E00045689C40A4B22C434460D8E70369194291
:1007F00014BF012000207047018370474183704778
:1008000010B4CB0800EB830001F00701046A8900F3
:100810000F238B4024EA03030362036A8A4042EAFF
:10082000030101625DF8044B704700BF29B9054A16
:10083000136B23EA000010637047024B1A6B1043DE
:10084000186370470038024029B9054A136C23EA3F
:10085000000010647047024B1A6C10431864704714
:100860000038024029B9054A536C23EA000050645D
:100870007047024B5A6C104358647047003802406E
:10088000F0B44A880F888D88CC880B894E893A430A
:100890002A4322438D89CC891A43324303882A4351
:1008A000224303F4415313439BB20380838B23F40D
:1008B00000631B041B0C83830B8A0382F0BC70470C
:1008C000002307220282038043808380C380038148
:1008D00043818381C3817047234A038890429BB23E
:1008E00012D002F5806290420ED0B0F1804F0BD052
:1008F000A2F58032904207D002F58062904203D088
:1009000002F58062904203D14A8823F070031343BA
:10091000164A904220D002F5806290421CD00A898B
:1009200023F440739BB2134303804B68C36210B43B
:100930000D4C0B880385A04207D00D4B984204D084
:10094000012383825DF8044B70478B7A0386012371
:1009500083825DF8044B704703804B68C3620B8849
:10096000038501238382704700000140001000408E
:100970000004014000234FF0FF32426003800381F6
:1009800043808372704700BF038829B923F00103B5
:100990001B041B0C038070479BB243F001030380D0
:1009A000704700BF83899BB21AB923EA0101818194
:1009B0007047194381817047038A828911EA0300D5
:1009C00092B203D0114214BF01200020704700BF33
:1009D000C94389B201827047838823F070031B04E6
:1009E0001B0C838083889BB219438180704700BFB2
:1009F0002DE9F04F2DED048BCF4C9FEDD07A85B0D3
:100A0000002602460290884604F500652346F2EC73
:100A1000017A5E6067EE877A083343ED027AAB4273
:100A20009FEDC78AF3D101230022C349C548DFF8EF
:100A30006C9305F08DFA4FF48072C349BE4805F0FF
:100A400093FEC24AD9F800101368C14801338B42A3
:100A5000136080F29F80D0ED005ABE4ADFEDB87A75
:100A600002F1F8011346B3EC017A994277EE877AE6
:100A7000F9D1B94BDFEDB26AB2EC017A9342E7EEFD
:100A8000076AF9D1B54BB64AC3ED006AB54B127887
:100A90001968B54EF4EEE56AF1EE10FAC4BFF0EE57
:100AA000665AC0ED006A8A4200F0188179DC96ED42
:100AB000007A9FEDA36AF6EE006A77EE666AF4EEBE
:100AC000C66AF1EE10FA40F26F81B2EE046A86EE69
:100AD000867A9FED9A6AC6ED006A37EE067A1A604A
:100AE0009FEDA25AA24B87EE856AB2EE045AF7EE4A
:100AF000007AE5EEC57A66EE265A26EE077A67EEAC
:100B0000A57A83ED006AB4EEE77A9A4BF1EE10FA1B
:100B1000C4BFF0EE477A83ED007A9FED897AD8BFA3
:100B2000C3ED007AF4EE476AF1EE10FA4AD1924A28
:100B300083ED007A1378F0EE477A002B46D18F4B85
:100B400003931946804A9FED8E6A002000230FE030
:100B500092ED007AB4EEE77AF1EE10FA15D8106053
:100B60000133B3F5007F02F1040201F1040144D026
:100B70007F2BEDDC92ED007A67EE066AB4EEE77A41
:100B8000F1EE10FAC1ED006AE9D937EE677A82ED2D
:100B9000007AE5E70023F0EE485A80ED008A136002
:100BA0005BE7D6ED006A9FED656AB6EE007A76EEF9
:100BB000876AB2EE045A86EE857AC6ED006A37EE91
:100BC000067A8CE76C4B1B78002BB8D0012B00F019
:100BD00090805D4B03F50062D3ED006A9FED587A7B
:100BE000F4EEE67AF1EE10FAB8BF36EEE77AA3EC4F
:100BF000017A9A42F0D1614B0393624FDFF848B11A
:100C0000DFED4F9AA7F1040ADAED010A17ED010AA8
:100C10009FED4B9AA0EEA90A04F058FBDBED008A89
:100C2000B0EE408A05F0CCFE68EE808AB0EE480A4D
:100C3000BBEC018A05F080FE28EE000A47ED018A30
:100C40000AF1080A0AED010AAA4507F10807DBD1F3
:100C5000039BDFF84CB183ED009A48484A4A5B4653
:100C6000802104F0DDFD494B1B78012B00F0A380AF
:100C700001231A463049334805F06AF9D6ED007A67
:100C8000434A4346B0EE007AF4EEC77AF1EE10FA2A
:100C90002168D8BF196004F10804CCBF1160D6EDFB
:100CA000007AAC4202F1040203F10403ECD1B0EE8D
:100CB000007AF4EEC77AF1EE10FA0ADD4FF4807391
:100CC0003449019300914346029A3149324805F074
:100CD000D3F905B0BDEC048BBDE8F08FD6ED006A0A
:100CE0009FED166AB2EE045A86EE857A37EE067AE2
:100CF000F6E6224B03931946134A9FED216A00231F
:100D000006E00133B3F5007F01F104013FF475AF54
:100D100092ED007ADFED0A6AF4EEC77AF1EE10FA8E
:100D200001DA77EE676A7F2BE2EC016AE9DC66EEB6
:100D3000866AC1ED006AE4E7F0460020CDCC4C3F66
:100D400000000000A89D0008E42E00202C020020D6
:100D500028020020EC2E00205C2F00204002002002
:100D6000D30A002020020020380200200000784230
:100D70003402002044020020381700200C4F0020CD
:100D800000004842F4460020E43A002034130020DA
:100D9000E42A0020E4260020D426002010010020B0
:100DA000E8420020CDCC4C3FF0EE466A1FED037ABE
:100DB00086ED006A93E63549D9F800000B68642295
:100DC000013302FB00F293420B60314B314A93ED49
:100DD000007A20DAD2ED007AB4EEE77AF1EE10FA7A
:100DE0002CDCF2EE086AF4EEE67AF1EE10FA40D46A
:100DF000DBF800302849DA1FF5EE006A082A0B609C
:100E000067EEA67A04D8B4EEE77AF1EE10FA2ADC9F
:100E100001F0A8F82CE7B4EEC97A0023F1EE10FA3D
:100E200082ED009A0B6009DCF0EE497ADBF80030C5
:100E30001949DA1F082A0B60E5D9E9E7DBF8003029
:100E4000D91F082912D8F2EE087AB4EEE77AF1EE4B
:100E500010FA82ED007A11D40F4AF5EE007A136091
:100E600067EE277ACFE701F059F801E70A4A1360E5
:100E7000CEE7B6EE009A67EE897AD7E7064AF6EE35
:100E8000007A136067EE277ABDE700BF3C020020BE
:100E9000E43A002024020020300200202DE9F04135
:100EA00001219CB080464448444E454D454FFFF7D4
:100EB000BDFC01214FF480700024FFF7D3FC4022D9
:100EC000032301A9404801928DF808308DF80B40AA
:100ED000FFF738FC3046FFF717FB3C4B0F934FF4FE
:100EE000806203F500710E9513924FF400634FF486
:100EF00000554FF480723046149315954FF400332B
:100F0000012516924FF400221793CDF844800D94DA
:100F10001094129418941A941B941995FFF7C2FB1D
:100F200029463046FFF7CAFB30460DA9FFF784FB80
:100F30002A4630461021FFF7E5FB29463046FFF7E9
:100F4000A7FB03A80394049405940694FFF71EFAE4
:100F500038464FF080524FF0C06307A909920A93B8
:100F600007948DF820408DF821400B948DF8305077
:100F7000FFF7E6F923462A4638460621FFF724FA0A
:100F800029463846FFF774FA29463846FFF766FACD
:100F900029463846FFF70EFA3822052368468DF8B1
:100FA00001508DF803508DF800208DF80230FFF7C6
:100FB0008FF91CB0BDE8F0810100400010640240D0
:100FC0004C2001400020014000000240F04200207F
:100FD00000B5012185B00846FFF736FC01A8FFF7F0
:100FE000C9FC002340F2747201A94FF080400292C4
:100FF000ADF80430ADF80C30ADF80630FFF76CFCFE
:1010000020214FF08040FFF7E7FC01214FF08040A6
:10101000FFF7BAFC05B05DF804FB00BFF0B5012195
:1010200097B005460846FFF701FC01214FF000503C
:10103000FFF70AFC01214FF400100024FFF7F6FB34
:101040002A4E2B488DF80B401022032301A9019250
:101050008DF80830FFF776FB24224FF4206303A9B4
:1010600020460392059304940694FFF70BFA30464A
:10107000FFF74AFA1F4B0B951F4A09934FF0606523
:1010800003F500710795089240274FF480634FF4F1
:1010900000654FF4005230460A970D930E954FF4B9
:1010A000003301250F924FF480774FF40022119303
:1010B0000C9412941494159410971395FFF7F2FA68
:1010C00029463046FFF7FAFA304607A9FFF7B4FA87
:1010D00029463046FFF7DCFA29462046FFF7FEF99D
:1010E00029462046FFF7E6F917B0F0BD88600240B8
:1010F00000000240E43600200874004070B500246F
:1011000082B04FF6E075244E244B254A20468DE8E8
:1011100030005A2103F096FD334601940095214A90
:10112000E121052003F08EFD3346019400951E4A0F
:10113000D2214FF4967003F085FD3346019400955B
:101140001A4ABE214FF4967003F07CFD3346019499
:101150000095174AAA214FF4967003F073FD3346A9
:1011600001940095134A96214FF4967003F06AFD9E
:10117000334601940095104A82214FF4967003F093
:1011800061FD0194009533460C4A6E214FF4967030
:1011900003F058FD02B070BD8001002088010020DE
:1011A0006C8700088C870008B4870008B88700089F
:1011B000BC870008C0870008C4870008C8870008EB
:1011C0002DE9F04194B001F01BF802F0B3FD0320CB
:1011D00003F0D4F900204FF6E07403F075F8002115
:1011E00000254E4E0094084655237D2203F048FF0B
:1011F0002946009455234FF4A072822003F040FF4B
:10120000334600940195464A464FDFF83C8105215C
:101210000A2003F017FD334601940095424A052148
:10122000162003F00FFD3346019400953F4A192123
:10123000162003F007FD3346019400953C4A2D210A
:10124000162003F0FFFC334601940095394A4121F2
:10125000162003F0F7FC33463A468DE830000521AE
:101260003C2003F0EFFC3A4633468DE8300019216C
:101270003C2003F0E7FC33468DE830002E4A2D2158
:101280003C2003F0DFFC33468DE830002B4A41213F
:101290003C2003F0D7FC28460094F0234FF4A072C2
:1012A000642103F0EDFEDE2340F23B126E210220AA
:1012B000009503F009FFFFF721FF214BDFF88CE0D9
:1012C00001950FCB0DF1080C8CE80F00BEE80F0064
:1012D00006AF0FC79EE803001A4B47F8040B39709E
:1012E0000FCB0DAF009487E80F00624633461921FB
:1012F000872003F0A7FC06AA43468DE830002D2185
:10130000872003F09FFC8DE8300043463A46412198
:10131000872003F097FC14B0BDE8F081880100201D
:10132000CC870008E0870008D0870008D487000831
:10133000D8870008DC870008E8870008F0870008E5
:10134000F88700082088000880010020088800082D
:1013500000B5012183B01020FFF768FA01220023B5
:101360006946064800928DF807208DF804308DF804
:101370000530FFF7E7F903B05DF804FB0010024009
:1013800010B4FCEEC07A83B0CDED017ABDF8044014
:10139000944203D303B05DF8044B7047091B89B234
:1013A0001A4603B05DF8044B02F04ABE07EE902ADD
:1013B000F8EE677A82B080EE270A07EE901AF8EE10
:1013C000677A20EE270AFCEEC07ACDED017ABDF8EF
:1013D0000420914201D9602A07D94FF6E07203F147
:1013E000780189B202B002F02BBEA2F140011F29A0
:1013F00009D9A2F120011F290DD9103A0F2A8CBF5B
:1014000000221F22EBE703F1780140F2FF7289B25C
:1014100002B002F015BE40F21D52E0E72DE9F043A4
:10142000B54B1C7895B064BBB44CB54D22682B68A5
:101430009A4234DDB34F3A780132D2B23A70B249AF
:10144000DFF8C0920DA806F02DFC4FF6E0780023DF
:1014500001930DAACDF80080AC4B05213C2003F090
:10146000F1FB3E78002E00F01781731E032B40F233
:101470000681042E00F2F68023682B6015B0BDE8CB
:10148000F083012C16D0022C00F0AF80032C39D051
:101490009A4B9B4D1B682B6015B0BDE8F0832DDA8D
:1014A000984F3B78002B00F02381013BDBB21A46BA
:1014B0003B70C4E7914C924D22682B689A4240F3EE
:1014C0000081934E3378022B9ABF0133DBB20323A2
:1014D0003370012B00F0B081022B00F0A081032BB0
:1014E000CAD14FF6E07200238DE80C001921874B1A
:1014F000884A3C2003F0A6FB2368BEE7BDD0814F9D
:101500003A789CE77D4C7E4D23682A68934200F32D
:101510004A81B2DA80490A780AB1013AD2B27F4BE5
:101520000A700FCB00270DAE86E80F0032460197F8
:101530000097764B0521872003F084FB3246019704
:101540000097724B1921872003F07CFB32460197EC
:1015500000976E4B2D21872003F074FB32460197D4
:1015600000976A4B4121872003F06CFB6C4BDFF83E
:10157000E0C101970FCB0DF1080888E80F00BCE827
:101580000F000DF1180EAEE80F009CE80300654B4C
:101590004EF8040B8EF800100FCB4FF6E07986E87A
:1015A0000F004246CDF80090584B1921872003F0D8
:1015B00049FB06AA0197CDF800905B4B2D218720AF
:1015C00003F040FB32460197CDF80090564B412185
:1015D000872003F037FB0197CDF800904B4B534A1F
:1015E00041213C2003F02EFB46E7444E444D336836
:1015F0002A68934240F3AE804D490F78002F7FF464
:101600003CAF4FF6E07801200197CDF800803F4BCA
:101610000870484A2D213C2003F014FBF0234FF4BE
:10162000A07264213846CDF8008003F029FD2046E1
:10163000DE2340F23B126E21009703F045FD334B51
:101640003D4A5A2138468DE8800103F0FBFA364BBB
:10165000CDF800800197394AE121052003F0F2FA24
:1016600033680AE74FF6E07200238DE80C0005218D
:10167000264B334A5B2003F0E5FA2368FDE64FF67C
:10168000E07200238DE80C000521204B2D4A5B20E1
:1016900003F0D8FA3E78ECE601961C4B2A4ACDF8C6
:1016A000008005213C2003F0CDFA0196CDF80080A2
:1016B000164B264A05216E2003F0C4FA99F8006003
:1016C000D3E680F2A780124E33780BB1013BDBB238
:1016D0003370002B7FF4FDAE4FF6E0728DE80C0006
:1016E00019210A4B184A3C2003F0ACFA3378F0E693
:1016F0001A463B70A3E600BF35130020CC0A002039
:101700003C170020D30A00207888000888010020B8
:10171000401B00209888000834130020A888000887
:10172000F88700082088000880010020F087000862
:1017300038170020A088000830880008508800086A
:101740008488000880880008E087000888870008EF
:1017500008880008BFF691AE3E490A78012A7FF456
:101760008CAE00274FF6E0780197CDF800803A4B19
:101770003A4A0F703C202D2103F064FA3846F023DA
:101780004FF4A0726421CDF8008003F079FCDE23D1
:10179000204640F23B126E21009703F095FCFFF7C4
:1017A000ADFC336869E62E4B01221A7000F060FB35
:1017B0002C4B0FCB00260DAF87E80F003A46264B87
:1017C000019605218720009603F03CFA3A46224B09
:1017D000019619218720009603F034FA3A461E4BF1
:1017E00001962D218720009603F02CFA3A461A4BD9
:1017F000019641218720009603F024FA4FF6E0730A
:101800008DE84800184A144B41213C2003F01AFA95
:10181000236832E63FF431AE144E337859E74FF681
:10182000E07200238DE80C0019210B4B104A3C207C
:1018300003F008FA337852E64FF6E07200238DE8A1
:101840000C001921044B0B4A3C2003F0FBF93378C0
:1018500042E600BF3817002088010020E887000812
:1018600034130020A8880008B8880008401B002016
:10187000908800088888000810B53B490B78022B37
:1018800082B025D900244FF6E0738DE81800374A5E
:10189000374B0C700A20052103F0D4F9344B354A3C
:1018A0000194009419210A2003F0CCF9304B314AFD
:1018B000019400942D210A2003F0C4F901940094AE
:1018C0002B4B2C4A41210A2003F0BCF902B010BD79
:1018D0000133DBB20024012B0B700194009425D05E
:1018E000022B244A224B4FF005014FF00A002AD068
:1018F00003F0A8F9019400941D4B1E4A19210A20F7
:1019000003F0A0F901940094194B1A4A2D210A20E2
:1019100003F098F94FF6E0738DE81800134A144B62
:1019200041210A2003F08EF902B010BD104B114A7C
:1019300005210A2003F086F94FF6E0738DE81800C0
:101940000A4A0B4BAEE703F07DF9094B094A0194B3
:10195000009419210A2003F075F94FF6E0738DE821
:101960001800024A024BA5E735130020CC87000877
:10197000880100208887000830B5174D85B0012107
:101980000220FEF761FF00244FF47A73284640F2EC
:10199000DC5201A90293ADF80420ADF80C40ADF87B
:1019A0000640FEF799FF012211462846FEF7FAFF8E
:1019B00028460121FEF7E8FF1D22012368468DF825
:1019C00001408DF802408DF800208DF80330FEF7BD
:1019D0007FFC05B030BD00BF0004004030B5154DA0
:1019E00085B001210820FEF72FFF0024124B02933F
:1019F000284601A9ADF80440ADF80C40ADF806400A
:101A0000FEF76AFF012211462846FEF7CBFF0121AF
:101A10000A48FEF7B9FF3222012368468DF80140DB
:101A20008DF802408DF800208DF80330FEF750FC51
:101A300005B030BD000C004020480100000400400B
:101A40002DE9F041294B2A4E2A4C356827688446F7
:101A50000FCB86B005EB85054FEA850EC7EB071760
:101A600002AD85E80F000EF1050E07F178084FF67C
:101A7000E07300271FFA8EF18DE8880062461E4B46
:101A80001FFA88F002F00EFE2368316803EB83032F
:101A90009B00B42B05DD0123194403293160236029
:101AA00016DD01EB810189003C290BDD00212A466E
:101AB00001910091012531600F4B256005218720A0
:101AC00003F0C0F823680133236006B0BDE8F0815D
:101AD00001EB81018900053189B201970097064B1E
:101AE0002A46872003F0AEF83168DAE7A8880008B4
:101AF000480200201401002088010020014B1868D2
:101B0000704700BF245F002008B501210448FEF79C
:101B100053FF18B1034A13680133136008BD00BFB7
:101B2000000C0040245F002000B583B04FF48074A7
:101B3000FFF746FB1F4B204A20480094192104F070
:101B40009DFB1F4B1F4A20480094652104F096FB23
:101B50001E4B1F4A1F480094112104F08FFB1E4B9F
:101B60001E4A1F480094112104F088FB9FED1D0AB6
:101B70001D4B1E4A1E480094202104F063FA2046A3
:101B8000FFF78CF92046FFF749FAFFF7E1FB194B05
:101B90001948802219460092402200F0F3FD0121ED
:101BA000154800F021FEFFF713FAFFF7E5FEFFF7F7
:101BB00015FFFEE7D40A0020EC840008004F002047
:101BC000601B002050850008185F00204C02002098
:101BD000E4860008F44E00208C06002028870008C8
:101BE0000C5700203333733F54220020D4210020AF
:101BF000D426002000040240441B0020034B1A8B13
:101C0000824200D07047184600F0F0BD441B00200F
:101C100010B5254C254823882549B3FA83F35B0981
:101C200000EB43204FF48072238003F011FD214B21
:101C30001B78032B1FD0022B25D0012B2BD093B167
:101C40001D491E48FEF7D4FE21881D4B1A4803EBA0
:101C500041214FF4807203F04BFD10211948BDE87B
:101C60001040FEF735BD4FF48073144A10491648F2
:101C700004F016FBE4E74FF48073104A0C49134854
:101C800004F00EFBDCE74FF480730C4A084910485F
:101C900004F006FBD4E74FF48073084A04490D486A
:101CA00004F0FEFACCE700BFD00A0020F04200208A
:101CB00040170020401B002038130020340F002064
:101CC000E436002010640240F44E0020185F00202B
:101CD000004F00200C5700202DE9F0472DED028B1E
:101CE000012182B05448FEF767FE20B902B0BDEC76
:101CF000028BBDE8F08701214F48FEF769FE4F4B8C
:101D00001B7843B3012B61D04D4A137833B1013BAB
:101D1000137002B0BDEC028BBDE8F087494D4A4C10
:101D200002232846137000F04DFD2B6847482360BE
:101D30000121FEF75BFD464B1870002843D0454B50
:101D400022681B689A42D1D002B0BDEC028BBDE87C
:101D5000F047FFF763BB404D404E414FDFED418AF6
:101D600005F5FE791624F5EC016A97ED007A96EDFB
:101D7000000ADFF8EC80C6EE877A20460023642252
:101D8000DC2167EEA87AFCEEE77ACDED017ABDF8AA
:101D900004E008EE10EAFFF7F3FAB8EE488A2046AE
:101DA0004FF6E073B0EE480A6422DC21FFF7E8FA50
:101DB0000234A945A6EC018AA4B2D4D12A4BD8F8A2
:101DC00000201A60A0E7FFF757FDB8E7224D244F27
:101DD000264E05F1FC091824D7ED007A3378DFF898
:101DE0008C80FCEEE77A2046CDED017AAA46BDF85C
:101DF0000420B5EC010A6421FFF7D8FAD7ED007A88
:101E00009AED000A3378FCEEE77AA01CCDED017A5A
:101E1000BDF8042080B26421FFF7C8FA04344D45B0
:101E2000A4B2D9D198F80030632B9ABF0133DBB24A
:101E30000023337068E700BF00040040381700201B
:101E400019010020441B0020CC0A00200010024091
:101E5000180100203C170020104F002010530020D4
:101E6000E43A00200000C842F04E0020D20A0020D0
:101E700018481949194ADFF89CC0F0B50123184FDA
:101E8000037013700B70174E174DDFF88CE0174C72
:101E90001748184A184903233B600F233360642313
:101EA0002B609623CCF80030CEF80030002323605E
:101EB00003601360114F124E124D134C1348144A15
:101EC0000B6002213B6033602B6023600360116074
:101ED000F0BD00BF740100206201002061010020FC
:101EE000700100206401002068010020F020002023
:101EF000F42000201021002008210020F8200020DC
:101F0000FC2000200C2100200421002000210020C2
:101F10001C0100206C0100207801002010B50C4B42
:101F20000C4C1A68002AC4BF00221A60236853B1FF
:101F3000094A0A4C0A48116800232370037009B942
:101F40000123136010BDFFF7D9FD2060F0E700BF4B
:101F5000F82000200821002000210020620100203C
:101F600074010020F8B5574C2368002B2BD0FFF7E5
:101F7000C5FD554E23683268544DC01AB0EB420F70
:101F8000286002DD524B1A78D2B1524C2368002BE4
:101F900007DDFFF7B3FD23684F4AC01A0023106026
:101FA00023604E4B1A7892B14D4C23783BB94D4A81
:101FB0002968126891422FDC474B00221A60F8BD55
:101FC00001221A70E1E7FFF799FD2060CFE745484D
:101FD000414C01682468A2F1AA3282FB0172A2EB93
:101FE000E172A242E0DC404F3A684FF0010E02FA83
:101FF0000EF2A1423A6083F800E01CDC33683B4AF1
:10200000234482FB0312A2EBE37203EBD37352006F
:102010005B1002603360C7E7334D2D492A680B70AF
:102020003F2A0BDC324B985CFFF70AFD01220023AC
:1020300022702B60C0E772443A60B5E7612A24D071
:102040000ADD732A2DD012DC652A26D06A2A20D117
:10205000284B2E221A70E9E74C2A2AD00FDD542A89
:1020600023D05E2A15D1234B2D221A70DEE77A2A5F
:1020700023D0F62A0DD11F4B24221A70D6E7472A07
:1020800007D11C4B3A221A70D0E71A4B27221A703C
:10209000CCE7184B23221A70C8E7164B40221A705F
:1020A000C4E7144B3F221A70C0E7124B21221A706A
:1020B000BCE7104B2C221A70B8E70E4B6B221A703B
:1020C000B4E700BFF82000206401002010210020A8
:1020D0006101002008210020F4200020740100206C
:1020E000620100207001002000210020ABAAAA2A72
:1020F000200100207C0100200649074A074B9A4234
:10210000BEBF51F8040B42F8040BF8E704488047BF
:1021100004480047E0B1000800000020040200204D
:1021200001220008E50100083349344A002301E098
:1021300041F8043B9142FBD3FFF7F6FCFEE7FEE7D4
:10214000FEE7FEE7FEE7FEE7FEE7FEE7FEE7FEE767
:10215000FEE7FEE7FEE7FEE7FEE7FEE7FEE7FEE757
:10216000FEE7FEE7FEE7FEE7FEE7FEE7FEE7FEE747
:10217000FEE7FEE7FEE7FEE7FEE7FEE7FEE7FEE737
:10218000FEE7FEE7FEE7FEE7FEE7FEE7FEE7FEE727
:10219000FEE7FEE7FEE7FEE7FEE7FEE7FEE7FEE717
:1021A000FEE7FEE7FEE7FEE7FEE7FEE7FEE7FEE707
:1021B000FEE7FEE7FEE7FEE7FEE7FEE7FEE7FEE7F7
:1021C000FEE7FEE7FEE7FEE7FEE7FEE7FEE7FEE7E7
:1021D000FEE7FEE7FEE7FEE7FEE7FEE7FEE7FEE7D7
:1021E000FEE7FEE7FEE7FEE7FEE7FEE7FEE7FEE7C7
:1021F000FEE7FEE7FEE7000004020020385F002053
:1022000039493A4BD1F88820394842F47002C1F874
:1022100088201A68002142F001021A6099601A6849
:1022200022F0847222F480321A6058601A6882B0F8
:1022300022F480221A60D960009101911A6842F458
:1022400080321A601A4603E0009BB3F5C06F09D0D4
:10225000136803F400330193009B01330093019B47
:10226000002BF1D0214B1B6813F4003318BF01235E
:102270000193019B012B05D01B4B4FF000629A602C
:1022800002B07047194B1B491A6C1B4842F0805230
:102290001A640A6842F480420A609A689A609A68EE
:1022A00042F400429A609A6842F4A0529A605860E0
:1022B0001A6842F080721A601A4611680B4B890145
:1022C000FBD50E4A40F2057111609A6822F00302B4
:1022D0009A609A6842F002029A601A46936803F084
:1022E0000C03082BFAD1C7E700ED00E000380240EC
:1022F000103000240070004019544007003C024098
:102300002DE9F041064684B015460C46A1B14B1E9E
:102310000B423FD0E70705D50121FFF7F1FF002869
:1023200040F0B780A00707D52A4602213046FFF7C4
:10233000E7FF002840F0AD80610700F1AE80220782
:1023400000F1B580E30600F1BC80A70600F1C38070
:10235000600600F19680210600F1C680E20500F1DA
:10236000CD80A30500F1D580670500F1DD80200553
:1023700000F1E580E10400F1FA80A20400F1EB80B5
:10238000630400F10081E30B40F00981002004B0F8
:10239000BDE8F081A24B1A680A427AD15B68194203
:1023A00077D1802900F0318100F21281082900F0F4
:1023B000208100F2FE80022900F02B81042900F028
:1023C0002681012965D10627012D00F0FF80002D0F
:1023D00014BF0022022200238DE80C0021461A4679
:1023E000304600F025FA204600F074FB5FFA80F8D2
:1023F00030468C4E00F038FB716C894B08F0FC02C3
:1024000002F1804202F59C3241F48041716408F08F
:102410000301966889004FF00F0E0EFA01FE26EABE
:102420000E0696609668C0B200FA01F131439160E1
:102430001968E243114019605968114059601968E0
:1024400021431960D9681140D9609968012D02EAC9
:1024500001029A6000F0B68015B1DA682243DA60B2
:102460009A6814439C600A22012303A88DF80C701B
:102470008DF80E808DF80D208DF80F30FDF728FFB8
:1024800084E72A4640213046FFF73AFF00283FF410
:1024900062AF012004B0BDE8F0812A460421304635
:1024A000FFF72EFF0028F4D122077FF54BAF2A4615
:1024B00008213046FFF724FF0028EAD1E3067FF524
:1024C00044AF2A4610213046FFF71AFF0028E0D11A
:1024D000A7067FF53DAF2A4620213046FFF710FFC3
:1024E00000283FF435AFD4E72A4680213046FFF775
:1024F00007FF0028CDD1E2057FF533AF2A464FF420
:1025000080713046FFF7FCFE0028C2D1A3057FF59D
:102510002BAF2A464FF400713046FFF7F1FE00283A
:10252000B7D167057FF523AF2A464FF48061304667
:10253000FFF7E6FE0028ACD120057FF51BAF2A4649
:102540004FF400613046FFF7DBFE0028A1D1E10423
:102550007FF513AF0BE02A464FF400513046FFF7EA
:10256000CFFE002895D163047FF50DAF0BE02A461E
:102570004FF480513046FFF7C3FE002889D1A204F2
:102580007FF5FEAEE7E72A464FF480413046FFF77D
:10259000B7FE00287FF47DAFE30B3FF4F7AE2A4689
:1025A00030464FF40041FFF7ABFE00283FF4EEAE9B
:1025B0006FE7202929D0402927D010297FF469AF5F
:1025C0000A2701E7DA681443DC604CE72A4602E791
:1025D000B1F5006F0BD00ED9B1F5005F07D01AD955
:1025E000B1F5804F03D0B1F5004F7FF452AF2827EB
:1025F000EAE60927E8E6B1F5007F06D0B1F5806F7D
:10260000F5D0B1F5807F7FF444AF1727DCE60827CB
:10261000DAE60727D8E6B1F5805FE8D039E700BFF2
:10262000003C01400038024008B5044B5A69D2070B
:1026300003D501205861FFF7E1FA08BD003C0140D5
:1026400008B5044B5A69920703D502205861FFF779
:10265000D5FA08BD003C014008B5044B5A69520741
:1026600003D504205861FFF7C9FA08BD003C0140BA
:1026700008B5044B5A69120703D508205861FFF7C3
:10268000BDFA08BD003C014008B5044B5A69D206AA
:1026900003D510205861FFF7B1FA08BD003C014096
:1026A00008B5174B5A69910625D4154B5A6952063D
:1026B0001CD4134B5A69100613D4114B5A69D10517
:1026C00009D40F4B5A69920504D54FF40070586134
:1026D000FFF794FA08BD4FF480705861FFF78EFA47
:1026E000EFE780205861FFF789FAE6E7402058615C
:1026F000FFF784FADDE720205861FFF77FFAD4E77F
:10270000003C014008B51E4B5A69500531D41C4BA2
:102710005A69110527D41A4B5A69D2041DD4184B93
:102720005A69900413D4164B5A69510409D4144BB6
:102730005A69120404D54FF400405861FFF75EFA5D
:1027400008BD4FF480405861FFF758FAEFE74FF4A7
:1027500000505861FFF752FAE5E74FF48050586196
:10276000FFF74CFADBE74FF400605861FFF746FAD9
:10277000D1E74FF480605861FFF740FAC7E700BF28
:10278000003C014070B582B00446BDF8185043616A
:102790000161012622836583084600251146022235
:1027A000FFF7AEFD618B606901952B462A460096C6
:1027B00000F03EF86572E56065602560A67202B0C3
:1027C00070BD00BFC368026803609A1A002B4260A4
:1027D00005DB14BF00230223037218467047012350
:1027E00003721846704700BF4172704710B4026907
:1027F000038B1269847A4169134014BF01220022BD
:102800009442096909D08272428B33B9437A1140EC
:1028100033B939B1C368013BC3605DF8044B7047FD
:102820000029F7D0C3685DF8044B0133C3607047DB
:10283000F0B49DF810709DF8146009B9F0BC7047B1
:102840000D462D49884238D02C4988422FD02C493A
:10285000884226D02B4988421DD02B49884244D03B
:102860002A4988423BD02A49884232D029498842A5
:1028700029D02949884204D1284C216B41F4807128
:102880002163274C2271A3712560E771667121468F
:10289000F0BCFDF757BF214C216B41F008012163CB
:1028A000E4E71E4C216B41F004012163DBE71B4C84
:1028B000216B41F002012163D2E7184C216B41F0FA
:1028C00001012163CCE7154C216B41F080012163AC
:1028D000D7E7124C216B41F040012163D1E70F4C47
:1028E000216B41F020012163CBE70C4C216B41F0BF
:1028F00010012163C5E700BF000002400004024050
:1029000000080240000C0240001002400014024087
:1029100000180240001C0240002002400038024023
:10292000142100202DE9F04F83B09DF830B09DF8C0
:10293000347011B903B0BDE8F08F99463F4B98420F
:102940005ED03F4B984255D03E4B98424CD03E4BC8
:10295000984243D03D4B98426AD03D4B984261D05B
:102960003C4B984258D03C4B98424FD03B4B9842FE
:1029700004D13B4C236B43F4807323638A4601925A
:10298000064600254FF001084AFA05F2D3070FD595
:1029900008FA05F4012C4FF0000105D06408012C61
:1029A00001F10101FAD189B23A463046FDF728FF1C
:1029B0000135102DE8D12B4A9DF804309371022483
:1029C00030461146C2F800A082F8079082F805B0A0
:1029D000147103B0BDE8F04FFDF7B4BE204C236B7B
:1029E00043F008032363BEE71D4C236B43F004034D
:1029F0002363B5E71A4C236B43F002032363ACE770
:102A0000174C236B43F001032363A6E7144C236B9D
:102A100043F080032363B1E7114C236B43F0400381
:102A20002363ABE70E4C236B43F020032363A5E73E
:102A30000B4C236B43F0100323639FE7000002401D
:102A40000004024000080240000C02400010024056
:102A50000014024000180240001C02400020024006
:102A60000038024014210020164A9042034623D029
:102A700002F58062904221D002F5806290421FD020
:102A800002F5806290420FD002F58062904211D030
:102A900000200D4A93420BD00C4A934206D00C4AB8
:102AA000934208BF082070470420F8E707207047CA
:102AB00006207047052070470120EAE70220E8E77A
:102AC0000320E9E70004024000180240001C024015
:102AD000002002400346012B4FF0000005D95B089F
:102AE0000130012B80B2FAD17047704738B5102100
:102AF000A948FDF781FE2021A748FDF77FFE0221AE
:102B0000A548FDF77BFEA54B012199811A46194680
:102B10001389A24C9D07FBD00B891806F8D402211B
:102B20009D48A389FDF768FE9D4B013BFDD1202107
:102B30009948FDF763FE02219748FDF75FFE974B2A
:102B4000CB2199811A4619461389944C9B07FBD0D7
:102B50000B891D06F8D402218F48A389FDF74CFE8E
:102B600020218D48FDF748FE02218B48FDF746FEE7
:102B700039232246A38121461389884C9807FBD02C
:102B80000B891B06F8D402218348A389FDF734FE84
:102B900020218148FDF730FE02217F48FDF72EFEFF
:102BA0002C232246A381214613897C4C9D07FBD010
:102BB0000D8905F08005ADB2002DF5D102217648D2
:102BC000A389FDF719FE20217348FDF715FE0221A8
:102BD0007148FDF713FE2246A581214613896F4CEB
:102BE0009807FBD00B891B06F8D402216A48A389F9
:102BF000FDF702FE20216848FDF7FEFD0221664830
:102C0000FDF7FCFD34232246A38121461389634C42
:102C10009D07FBD00B891806F8D402215E48A389D2
:102C2000FDF7EAFD20215C48FDF7E6FD02215A4848
:102C3000FDF7E4FD02232246A38121461389574C68
:102C40009B07FBD00B891D06F8D402215248A389AB
:102C5000FDF7D2FD20215048FDF7D0FD02214E485E
:102C6000FDF7CCFDCF232246A381214613894B4C8F
:102C70009807FBD00D8905F08005ADB2002DF5D188
:102C800002214548A389FDF7B7FD20214248FDF701
:102C9000B3FD02214048FDF7B1FD2246A581214642
:102CA00013893E4C9B07FBD00B891D06F8D40221EB
:102CB0003948A389FDF7A0FD20213748FDF79CFD89
:102CC00002213548FDF79AFDC1232246A381214602
:102CD0001389324C9807FBD00B891B06F8D40221CC
:102CE0002D48A389FDF788FD20212B48FDF784FDA1
:102CF00002212948FDF782FD30232246A381214687
:102D00001389264C9D07FBD00B891806F8D40221A5
:102D10002148A389FDF770FD20211F48FDF76EFDB6
:102D200002211D48FDF76AFDE8232246A3812146C2
:102D300013891A4C9B07FBD00B891D06F8D402217E
:102D40001548A389FDF758FD20211348FDF754FDD0
:102D500002211148FDF752FD85232246A381214619
:102D600013890E4C9807FBD00D8905F08005ADB294
:102D7000002DF5D102210848A389FDF73DFD202152
:102D80000548FDF739FD02210348FDF737FD2246CE
:102D9000A581214606E000BF000C0240003C004037
:102DA00080841E001389AA4C9B07FBD00B891D064B
:102DB000F8D40221A748A389FDF71EFD2021A548CC
:102DC000FDF71AFD0221A348FDF718FD78232246DE
:102DD000A381214613899E4C9807FBD00B891B06C3
:102DE000F8D402219B48A389FDF706FD20219948CC
:102DF000FDF704FD02219748FDF700FDEA23224676
:102E0000A38121461389924C9D07FBD00D8905F0C3
:102E10008005ADB2002DF5D102218E48A389FDF7C2
:102E2000EBFC20218B48FDF7E7FC02218948FDF7E8
:102E3000E5FC2246A58121461389854C9807FBD0E5
:102E40000D8905F08005ADB2002DF5D10221814834
:102E5000A389FDF7D1FC20217E48FDF7CDFC02219E
:102E60007C48FDF7CBFC2246A58121461389784C8E
:102E70009B07FBD00B891D06F8D402217548A38956
:102E8000FDF7BAFC20217348FDF7B8FC0221714818
:102E9000FDF7B4FCED232246A381214613896C4C37
:102EA0009807FBD00B891B06F8D402216948A38937
:102EB000FDF7A2FC20216748FDF79EFC0221654832
:102EC000FDF79CFC64232246A38121461389604CB4
:102ED0009D07FBD00B891806F8D402215D48A38911
:102EE000FDF78AFC20215B48FDF786FC022159484A
:102EF000FDF784FC03232246A38121461389544C09
:102F00009B07FBD00B891D06F8D402215148A389E9
:102F1000FDF772FC20214F48FDF76EFC02214D4861
:102F2000FDF76CFC12232246A38121461389484CED
:102F30009807FBD00B891B06F8D402214548A389CA
:102F4000FDF75AFC20214348FDF756FC0221414879
:102F5000FDF754FC81232246A381214613893C4C72
:102F60009D07FBD00B891806F8D402213948A389A4
:102F7000FDF742FC20213748FDF740FC022135488F
:102F8000FDF73CFCF7232246A38121461389304CF0
:102F90009B07FBD00B891D06F8D402212D48A3897D
:102FA000FDF72AFC20212B48FDF726FC02212948A9
:102FB000FDF724FC20232246A38121461389244CBB
:102FC0009807FBD00B891B06F8D402212148A3895E
:102FD000FDF712FC20211F48FDF710FC02211D48BF
:102FE000FDF70CFCC0232246A38121461389184C0F
:102FF0009D07FBD00B891806F8D402211548A38938
:10300000FDF7FAFB20211348FDF7F6FB02211148DA
:10301000FDF7F4FB23232246A381214613890C4CA0
:103020009B07FBD00B891D06F8D402210948A38910
:10303000FDF7E2FB20210748FDF7E0FB02210548F0
:10304000FDF7DCFBC1232246A381214604E000BF3B
:10305000003C0040000C02401389A94C9807FBD0AB
:103060000B891B06F8D40221A648A389FDF7C4FBEF
:103070002021A448FDF7C0FB0221A248FDF7BEFBBA
:1030800010232246A381214613899D4C9D07FBD026
:103090000B891806F8D402219A48A389FDF7ACFBE6
:1030A00020219848FDF7AAFB02219648FDF7A6FBD0
:1030B000C5232246A38121461389914C9B07FBD04F
:1030C0000B891D06F8D402218E48A389FDF794FBD5
:1030D00020218C48FDF790FB02218A48FDF78EFBEA
:1030E0003E232246A38121461389854C9807FBD0B5
:1030F0000B891B06F8D402218248A389FDF77CFBCB
:1031000020218048FDF778FB02217E48FDF776FB01
:1031100028232246A38121461389794C9D07FBD0A1
:103120000B891806F8D402217648A389FDF764FBC1
:1031300020217448FDF762FB02217248FDF75EFB17
:10314000C7232246A381214613896D4C9B07FBD0E0
:103150000B891D06F8D402216A48A389FDF74CFBB0
:1031600020216848FDF748FB02216648FDF746FB31
:1031700086232246A38121461389614C9807FBD000
:103180000B891B06F8D402215E48A389FDF734FBA6
:1031900020215C48FDF732FB02215A48FDF72EFB47
:1031A00036232246A38121461389554C9D07FBD027
:1031B0000B891806F8D402215248A389FDF71CFB9D
:1031C00020215048FDF718FB02214E48FDF716FB61
:1031D00048232246A38121461389494C9B07FBD0F3
:1031E0000B891D06F8D402214648A389FDF704FB8C
:1031F00020214448FDF702FB02214248FDF7FEFA78
:103200003A232246A381214613893D4C9807FBD0DF
:103210000B891B06F8D402213A48A389FDF7ECFA82
:1032200020213848FDF7E8FA02213648FDF7E6FA92
:1032300055232246A38121461389314C9D07FBD09B
:103240000B891806F8D402212E48A389FDF7D4FA79
:1032500020212C48FDF7D2FA02212A48FDF7CEFAA8
:10326000B1232246A38121461389254C9B07FBD01D
:103270000D8905F08005ADB2002DF5D10221214860
:10328000A389FDF7B9FA20211E48FDF7B5FA0221FE
:103290001C48FDF7B3FA2246A58121461389184C34
:1032A0009D07FBD00B891806F8D402211548A38985
:1032B000FDF7A2FA20211348FDF79EFA02211148DA
:1032C000FDF79CFA18232246A381214613890C4C52
:1032D0009B07FBD00B891D06F8D402210948A3895E
:1032E000FDF78AFA20210748FDF788FA02210548F0
:1032F000FDF784FAB6232246A381214604E000BFED
:10330000003C0040000C02401389A84C9807FBD0F9
:103310000B891B06F8D40221A548A389FDF76CFA96
:103320002021A348FDF768FA0221A148FDF766FABB
:1033300008232246A381214613899C4C9D07FBD07C
:103340000B891806F8D402219948A389FDF754FA8D
:1033500020219748FDF750FA02219548FDF74EFAD3
:1033600082232246A38121461389904C9B07FBD0E0
:103370000B891D06F8D402218D48A389FDF73CFA7C
:1033800020218B48FDF738FA02218948FDF736FAEB
:1033900027232246A38121461389844C9807FBD01A
:1033A0000B891B06F8D402218148A389FDF724FA72
:1033B00020217F48FDF722FA02217D48FDF71EFA01
:1033C000F2232246A38121461389784C9D07FBD026
:1033D0000D8905F08005ADB2002DF5D102217448AC
:1033E000A389FDF709FA20217148FDF705FA0221AA
:1033F0006F48FDF703FA2246A581214613896B4CDD
:103400009807FBD00B891B06F8D402216848A389D2
:10341000FDF7F2F920216648FDF7F0F90221644832
:10342000FDF7ECF92A232246A381214613895F4C3C
:103430009D07FBD00D8905F08005ADB2002DF5D1BB
:1034400002215B48A389FDF7D7F920215848FDF7F1
:10345000D3F902215648FDF7D1F92246A58121462C
:103460001389524C9807FBD00D8905F08005ADB249
:10347000002DF5D102214E48A389FDF7BDF9202189
:103480004B48FDF7B9F902214948FDF7B7F9224643
:10349000A58121461389454C9B07FBD00D8905F07A
:1034A0008005ADB2002DF5D102214148A389FDF779
:1034B000A3F920213E48FDF79FF902213C48FDF782
:1034C0009DF92246A58121461389384C9D07FBD0E2
:1034D0000B891806F8D402213548A389FDF78CF929
:1034E00020213348FDF788F902213148FDF786F99C
:1034F000EF232246A381214613892C4C9B07FBD046
:103500000B891D06F8D402212948A389FDF774F917
:1035100020212748FDF772F902212548FDF76EF9B1
:103520002B232246A38121461389204C9807FBD0E8
:103530000D8905F08005ADB2002DF5D102211C48A2
:10354000A389FDF759F920211948FDF755F9022102
:103550001748FDF753F92246A58121461389134CDC
:103560009B07FBD00D8905F08005ADB2002DF5D18C
:1035700002210F48A389FDF73FF920210C48FDF7F0
:103580003BF902210A48FDF739F92246A581214677
:103590001389064C9D07FBD00B891806F8D402212D
:1035A0000348A389FDF728F9202103E0003C0040EF
:1035B000000C0240A948FDF71FF90221A748FDF7BA
:1035C0001DF901232246A38121461389A44C9B07A0
:1035D000FBD00B891D06F8D40221A048A389FDF772
:1035E0000BF920219D48FDF707F902219B48FDF7C3
:1035F00005F93F232246A38121461389984C980759
:10360000FBD00B891B06F8D402219448A389FDF74F
:10361000F3F820219148FDF7F1F802218F48FDF7DA
:10362000EDF826232246A381214613898C4C9D0761
:10363000FBD00B891806F8D402218848A389FDF72E
:10364000DBF820218548FDF7D7F802218348FDF7F4
:10365000D5F801232246A38121461389804C9B077C
:10366000FBD00B891D06F8D402217C48A389FDF705
:10367000C3F820217948FDF7C1F802217748FDF70A
:10368000BDF8E0232246A38121461389744C980794
:10369000FBD00B891B06F8D402217048A389FDF7E3
:1036A000ABF820216D48FDF7A7F802216B48FDF724
:1036B000A5F80F232246A38121461389684C9D0754
:1036C000FBD00B891806F8D402216448A389FDF7C2
:1036D00093F820216148FDF78FF802215F48FDF73C
:1036E0008DF831232246A381214613895C4C9B0728
:1036F000FBD00B891D06F8D402215848A389FDF799
:103700007BF820215548FDF777F802215348FDF753
:1037100075F82B232246A38121461389504C980724
:10372000FBD00B891B06F8D402214C48A389FDF776
:1037300063F820214948FDF75FF802214748FDF76B
:103740005DF80C232246A38121461389444C9D0732
:10375000FBD00B891806F8D402214048A389FDF755
:103760004BF820213D48FDF747F802213B48FDF783
:1037700045F80E232246A38121461389384C9B0726
:10378000FBD00B891D06F8D402213448A389FDF72C
:1037900033F820213148FDF72FF802212F48FDF79B
:1037A0002DF808232246A381214613892C4C980723
:1037B000FBD00B891B06F8D402212848A389FDF70A
:1037C0001BF820212548FDF717F802212348FDF7B3
:1037D00015F84E232246A38121461389204C9D07CC
:1037E000FBD00B891806F8D402211C48A389FDF7E9
:1037F00003F820211948FCF7FFFF02211748FCF7C6
:10380000FDFFF1232246A38121461389144C9B0717
:10381000FBD00B891D06F8D402211048A389FCF7C0
:10382000EBFF20210D48FCF7E7FF02210B48FCF7D6
:10383000E5FF37232246A38121461389084C9807C8
:10384000FBD00B891B06F8D402210448A389FCF79E
:10385000D3FF20210148FCF7CFFF03E0000C02401A
:10386000003C00400221A848FCF7C8FF072322467D
:10387000A38121461389A54C9D07FBD00B8918060F
:10388000F8D40221A048A389FCF7B6FF20219E4866
:10389000FCF7B2FF02219C48FCF7B0FF1023224640
:1038A000A38121461389994C9B07FBD00B891D06E8
:1038B000F8D402219448A389FCF79EFF2021924866
:1038C000FCF79AFF02219048FCF798FF0323224659
:1038D000A381214613898D4C9807FBD00B891B06C9
:1038E000F8D402218848A389FCF786FF2021864866
:1038F000FCF782FF02218448FCF780FF0E2322465A
:10390000A38121461389814C9D07FBD00B891806A2
:10391000F8D402217C48A389FCF76EFF20217A4865
:10392000FCF76AFF02217848FCF768FF092322466A
:10393000A38121461389754C9B07FBD00D8905F0A7
:103940008005ADB2002DF5D102216F48A389FCF7A7
:1039500053FF20216C48FCF74FFF02216A48FCF717
:103960004DFF2246A58121461389684C9D07FBD057
:103970000B891806F8D402216348A389FCF73CFFA1
:1039800020216148FCF73AFF02215F48FCF736FF2F
:10399000E1232246A381214613895C4C9B07FBD07F
:1039A0000D8905F08005ADB2002DF5D102215648F4
:1039B000A389FCF721FF20215348FCF71DFF0221BA
:1039C0005148FCF71BFF2246A581214613894F4C25
:1039D0009D07FBD00B891806F8D402214A48A38919
:1039E000FCF70AFF20214848FCF706FF0221464861
:1039F000FCF704FF0E232246A38121461389434C82
:103A00009B07FBD00B891D06F8D402213E48A389F1
:103A1000FCF7F2FE20213C48FCF7EEFE02213A487A
:103A2000FCF7ECFE14232246A38121461389374C70
:103A30009807FBD00B891B06F8D402213248A389D2
:103A4000FCF7DAFE20213048FCF7D6FE02212E4892
:103A5000FCF7D4FE03232246A381214613892B4C75
:103A60009D07FBD00B891806F8D402212648A389AC
:103A7000FCF7C2FE20212448FCF7BEFE02212248AA
:103A8000FCF7BCFE11232246A381214613891F4C5B
:103A90009B07FBD00B891D06F8D402211A48A38985
:103AA000FCF7AAFE20211848FCF7A6FE02211648C2
:103AB000FCF7A4FE07232246A38121461389134C59
:103AC0009807FBD00B891B06F8D402210E48A38966
:103AD000FCF792FE20210C48FCF78EFE02210A48DA
:103AE000FCF78CFE31232246A38121461389074C23
:103AF0009D07FBD00B891806F8D402210248A38940
:103B0000FCF77AFE202103E0000C0240003C00405C
:103B10008548FCF771FE02218348FCF76FFEC12344
:103B20002246A38121461389804C9B07FBD00B8939
:103B30001D06F8D402217C48A389FCF75DFE2021F4
:103B40007948FCF759FE02217748FCF757FE4823D5
:103B50002246A38121461389744C9807FBD00B8918
:103B60001B06F8D402217048A389FCF745FE2021EA
:103B70006D48FCF741FE02216B48FCF73FFE08232D
:103B80002246A38121461389684C9D07FBD00B89EF
:103B90001806F8D402216448A389FCF72DFE2021E1
:103BA0006148FCF729FE02215F48FCF727FE0F233E
:103BB0002246A381214613895C4C9B07FBD00B89CD
:103BC0001D06F8D402215848A389FCF715FE2021D0
:103BD0005548FCF711FE02215348FCF70FFE0C2359
:103BE0002246A38121461389504C9807FBD00B89AC
:103BF0001B06F8D402214C48A389FCF7FDFD2021C7
:103C00004948FCF7F9FD02214748FCF7F7FD31234D
:103C10002246A38121461389444C9D07FBD00B8982
:103C20001806F8D402214048A389FCF7E5FD2021BD
:103C30003D48FCF7E1FD02213B48FCF7DFFD362360
:103C40002246A38121461389384C9B07FBD00B8960
:103C50001D06F8D402213448A389FCF7CDFD2021AC
:103C60003148FCF7C9FD02212F48FCF7C7FD0F239F
:103C70002246A381214613892C4C9807FBD00B893F
:103C80001B06F8D402212848A389FCF7B5FD2021A2
:103C90002548FCF7B3FD02212348FCF7AFFD1123B3
:103CA0002246A38121461389204C9D07FBD00B8916
:103CB0001806F8D402211C48A389FCF79DFD1C4B73
:103CC000013BFDD120211848FCF798FD0221164840
:103CD000FCF794FD154B292199811A461946138941
:103CE000124C9B07FBD00B891D06F8D402210E480D
:103CF000A389FCF781FD20210B48FCF77FFD022101
:103D00000948FCF77BFD2C232246A3812146138919
:103D1000064C9807FBD00B891B06F8D402210248F9
:103D2000A389FCF769FD38BD000C0240003C00404F
:103D300040420F00F0B5002483B003278DE89000C7
:103D4000234601222021AD48AD4EFEF771FD012230
:103D500015468DE8900023460221A848FEF768FD2D
:103D600023462A4601971021A4480095FEF760FDDE
:103D70000221A248FCF740FD2946304601F0BEF979
:103D8000FEF7B4FE9F4AA049A04B9C4814800C80CB
:103D90004FF4A0722021F0275A801D711F80FCF77C
:103DA0002DFD02219548FCF729FD2A233246B381D7
:103DB00031461389924C9E07FBD00D8905F0800592
:103DC000ADB2002DF5D102218C48A389FCF714FD7A
:103DD00020218A48FCF710FD02218848FCF70EFDDF
:103DE0002246A58121461389854C9D07FBD00D896C
:103DF00005F08005ADB2002DF5D102217F48A389E1
:103E0000FCF7FAFC20217D48FCF7F6FC02217B48F8
:103E1000FCF7F4FC2246A58121461389784C9807CB
:103E2000FBD00D8905F08005ADB2002DF5D1022142
:103E30007248A389FCF7E0FC20217048FCF7DCFC09
:103E400002216E48FCF7DAFC2246A581214613893F
:103E50006B4C9B07FBD00B891F06F8D402216748E7
:103E6000A389FCF7C9FC20216448FCF7C5FC0221AA
:103E70006248FCF7C3FCEF232246A3812146138945
:103E80005F4C9E07FBD00B891D06F8D402215B48CE
:103E9000A389FCF7B1FC20215848FCF7AFFC0221B4
:103EA0005648FCF7ABFC2B232246A38121461389FD
:103EB000534C9807FBD00D8905F08005ADB2002D5D
:103EC000F5D102214D48A389FCF796FC20214B48EF
:103ED000FCF792FC02214948FCF790FC2246A581A0
:103EE00021461389464C9B07FBD00D8905F08005C0
:103EF000ADB2002DF5D102214048A389FCF77CFC2E
:103F000020213E48FCF778FC02213C48FCF776FC77
:103F10002246A58121461389394C9F07FBD00B8986
:103F20001E06F8D402213548A389FCF765FC202140
:103F30003248FCF761FC02213048FCF75FFC0123AA
:103F40002246A381214613892D4C9D07FBD00B8966
:103F50001806F8D402212948A389FCF74DFC20213A
:103F60002648FCF749FC02212448FCF747FC3F2384
:103F70002246A38121461389214C9B07FBD00B8944
:103F80001F06F8D402211D48A389FCF735FC202127
:103F90001A48FCF733FC02211848FCF72FFC2C23AD
:103FA0002246A38121461389154C9E07FBD00B891D
:103FB0001D06F8D402211148A389FCF71DFC2746F1
:103FC00026464FF4963520210C48FCF715FC0221BB
:103FD0000A48FCF713FCFF23A38123899807FCD030
:103FE0003B891906F9D402210448B389FCF704FC83
:103FF00020210248FCF700FC0AE000BF000C024050
:10400000003C0040325F0020285F00202C5F002031
:1040100002210A48FCF7F2FBFF23B38123899A07A8
:10402000FCD03B891B06F9D402210448B389FCF774
:10403000E3FB013DC7D103B0F0BD00BF000C02405F
:104040002DE9F04107460D469D4820211446FCF716
:10405000D5FB02219A48FCF7D1FB9A4B2A21998182
:104060001A4619461389974E9807FBD00B891B06F1
:10407000F8D402219248B389FCF7BEFB2021904876
:10408000FCF7BAFB4FEA172802218D48FCF7B6FB74
:104090003246A6F80C80314613898A4E9807FBD029
:1040A0000B891B06F8D402218548B389FCF7A4FBD1
:1040B00020218348FCF7A0FBFFB202218048FCF7D7
:1040C0009DFB3246B781314613897E4E9807FBD05F
:1040D0000B891B06F8D402217948B389FCF78CFBC5
:1040E00020217748FCF788FB02217548FCF786FB06
:1040F0003246A6F80C8031461389724E9807FBD0E1
:104100000B891B06F8D402216D48B389FCF774FBB8
:1041100020216B48FCF770FB02216948FCF76EFB1D
:104120003246B78131461389664E9F07FBD00B8913
:104130001806F8D402216248B389FCF75DFB202100
:104140005F48FCF75BFB02215D48FCF757FB2B2324
:104150003246B381314613895A4E9B07FBD00B89F7
:104160001F06F8D402215648B389FCF745FB2021ED
:104170005348FCF741FB2F0A02215148FCF73EFB54
:104180003246B781314613894E4E9807FBD00B89D2
:104190001B06F8D402214A48B389FCF72DFB2021E5
:1041A0004748FCF729FBEDB202214548FCF726FB06
:1041B0003246B58131461389424E9807FBD00B89B0
:1041C0001B06F8D402213E48B389FCF715FB2021D9
:1041D0003B48FCF711FB02213948FCF70FFB324644
:1041E000B78131461389374E9807FBD00B891B06E0
:1041F000F8D402213248B389FCF7FEFA2021304876
:10420000FCF7FAFA02212E48FCF7F8FA3246B5819B
:10421000314613892B4D9F07FBD00B891E06F8D41E
:1042200002212748AB89FCF7E7FA20212448FCF754
:10423000E5FA02212248FCF7E1FA2C232A46AB8159
:10424000294613891F4D9807FBD00B891B06F8D40C
:1042500002211B48AB89FCF7CFFA20211848FCF754
:10426000CBFA02211648FCF7C9FAC4F307232A4601
:10427000AB8129461389134D9F07FBD00B891E067E
:10428000F8D402210E48AB89FCF7B6FA20210C487D
:10429000FCF7B2FAE4B20A480221FCF7AFFA2A4668
:1042A000AC812846138907499C07FBD003891B066C
:1042B000F8D48B8902480221BDE8F041FCF79CBA92
:1042C000000C0240003C00402DE9F843A84B80461A
:1042D0002021A8481D885C88FCF790FA0221A54897
:1042E000FCF78CFAA44B2A21013D013C9981ADB227
:1042F000A4B21A4619464FEA182913899E4E9B0705
:10430000FBD00F8907F08007BFB2002FF5D1022143
:104310009848B389FCF770FA20219648FCF76CFAAC
:1043200002219448FCF76AFA3246B7813146138974
:10433000914E9F07FBD00F8907F08007BFB2002F77
:10434000F5D102218B48B389FCF756FA2021894820
:10435000FCF752FA02218748FCF750FA3246B7813F
:1043600031461389844E9807FBD00B891B06F8D47D
:1043700002218048B389FCF73FFA20217D48FCF7F1
:104380003BFA02217B48FCF739FA2B0A3246B3810B
:1043900031461389784E9F07FBD00B891806F8D455
:1043A00002217448B389FCF727FA20217148FCF7F1
:1043B00023FAEDB202216F48FCF720FA3246B581AC
:1043C000314613896C4D9B07FBD00B891F06F8D42F
:1043D00002216848AB89FCF70FFA20216548FCF7F9
:1043E0000DFA02216348FCF709FA2B232A46AB8118
:1043F00029461389604D9E07FBD00E8906F0800682
:10440000B6B2002EF5D102215A48AB89FCF7F4F977
:1044100020215848FCF7F0F902215648FCF7EEF944
:104420002A46AE8129461389534D9807FBD00E8941
:1044300006F08006B6B2002EF5D102214D48AB89B8
:10444000FCF7DAF920214B48FCF7D6F9022149485C
:10445000FCF7D4F92A46AE8129461389464D9B07BD
:10446000FBD00B891F06F8D402214248AB89FCF728
:10447000C3F920213F48FCF7BFF902213D48FCF772
:10448000BDF9230A2A46AB81294613893A4D9E0776
:10449000FBD00B891806F8D402213648AB89FCF70B
:1044A000ABF920213348FCF7A7F9E4B202213148E7
:1044B000FCF7A4F92A46AC81294613892E4C9B07A8
:1044C000FBD00B891F06F8D402212A48A389FCF7E8
:1044D00093F920212748FCF791F902212548FCF7A0
:1044E0008DF92C232246A38121461389224C9E0755
:1044F000FBD00B891D06F8D402211E48A389FCF7C6
:104500007BF95FFA89F95FFA88F8254627464FF468
:10451000963620211748FCF76FF902211548FCF761
:104520006DF9A4F80C9023899807FCD02B89190603
:10453000F9D402210F48BB89FCF75EF920210D4810
:10454000FCF75AF902210B48FCF758F9A7F80C8040
:1045500023899A07FCD02B891B06F9D40221054830
:10456000BB89FCF749F9013ED3D1BDE8F88300BF10
:104570002C5F0020000C0240003C004038B5202198
:1045800005464548FCF73AF902214348FCF736F95D
:10459000424B362199811A46194613893F4C980798
:1045A000FBD00B891B06F8D402213B48A389FCF7FA
:1045B00023F975B1012D46D0022D58D0032D29D0F5
:1045C000374B4FF4A070F0210022188059801A71E7
:1045D00038BD20213048FCF70FF902212E48FCF7A6
:1045E0000DF958232246A381214613892B4C9807A5
:1045F000FBD00B891B06F8D402212748A389FCF7BE
:10460000FBF8274BF0204FF4A0710122188059804D
:104610001A7138BD20212048FCF7EEF802211E480F
:10462000FCF7ECF8E8232246A381214613891B4CB2
:104630009807FBD00B891B06F8D402211648A389E2
:10464000FCF7DAF8BCE720211348FCF7D5F8022183
:104650001148FCF7D3F888232246A3812146138909
:104660000E4C9D07FBD00B891806F8D4C4E7202117
:104670000948FCF7C1F829460748FCF7BFF828238A
:104680002246A38121461389044C9B07FBD00B894A
:104690001D06F8D4D1E700BF000C0240003C0040EA
:1046A0002C5F00202DE9F04FB34DB44C2880B44D61
:1046B000248829801D784619A64287B040F3B98224
:1046C0005878AF4C08442080AB48002101801D7809
:1046D0005E78002E00F077810293A2F1200305930B
:1046E000109BDFF8A482C3F307230493119BC3F349
:1046F000072303930023C24644460193019A059B76
:1047000003FB0623029A526832F813B0002D00F022
:10471000548100260BFA06F31A0400F15A81119B0A
:10472000002BC0F24481964B96481F88019B8D193F
:1047300020211F44FCF762F802219248FCF75EF842
:104740002A23ADB2BFB2A8F80C30B8F808309907E8
:10475000FBD0BAF808301A06F7D402218948A38999
:10476000FCF74AF820218748FCF746F84FEA15295C
:1047700002218448FCF742F8A4F80C90B8F80830FD
:104780009B07FBD0BAF808301806F7D402217D4801
:10479000A389FCF731F820217A48FCF72DF8EDB217
:1047A00002217848FCF72AF8A581B8F80830990763
:1047B000FBD0BAF808301A06F7D402217148A38951
:1047C000FCF71AF820216F48FCF716F802216D4813
:1047D000FCF714F8A4F80C90B8F808309B07FBD04D
:1047E000BAF808301806F7D402216648A389FCF706
:1047F00003F820216348FBF7FFFF02216148FBF724
:10480000FDFFA581B8F808309907FBD0BAF8083049
:104810001A06F7D402215B48A389FBF7EDFF20219C
:104820005848FBF7EBFF02215648FBF7E7FF2B2325
:10483000A381B8F808309B07FBD0BAF808301D06F2
:10484000F7D402214F48A389FBF7D6FF20214D481A
:10485000FBF7D2FF3D0A02214A48FBF7CFFFA581B3
:10486000B8F808309807FBD0BAF808301906F7D422
:1048700002214448A389FBF7BFFF20214148FBF7F1
:10488000BBFFFFB202213F48FBF7B8FFA781B8F892
:1048900008309A07FBD0BAF808301B06F7D402217B
:1048A0003848A389FBF7A8FF20213648FBF7A4FF6F
:1048B00002213448FBF7A2FFA581B8F80830980719
:1048C000FBD0BAF808301906F7D402212D48A38985
:1048D000FBF792FF20212B48FBF78EFF022129488E
:1048E000FBF78CFFA781B8F808309A07FBD0BAF81D
:1048F00008301B06F7D402212248A389FBF77CFF6E
:1049000020212048FBF77AFF02211E48FBF776FFA3
:104910002C23A381B8F808309F07FBD0BAF80830E1
:104920001D06F7D402211748A389FBF765FF202154
:104930001448FBF761FF02211248FBF75FFFBDF847
:104940000C30A381B8F808309807FBD0BAF80830CB
:104950001906F7D402210B48A389FBF74DFF20214C
:104960000848FBF749FF02210648FBF747FF9DF87F
:104970004430A3810AE000BF285F00202C5F0020A4
:10498000325F0020000C0240003C0040B8F80830C4
:104990009A07FBD0BAF808301B06F7D40221A648C4
:1049A000A389FBF729FF029B1D78A44B19880136C8
:1049B000B5423FF6AFAE029B5E78019B01339E424B
:1049C00001933FF69BAE9D4B2944198007B0BDE88B
:1049D000F08F9B4B98481F88019B8D1920211F4405
:1049E000FBF70CFF02219448FBF708FF2A23ADB226
:1049F000BFB2A8F80C30B8F808309B07FBD0BAF863
:104A000008301806F7D402218B48A389FBF7F4FE7F
:104A100020218948FBF7F0FE4FEA1529022186483C
:104A2000FBF7ECFEA4F80C90B8F808309907FBD01F
:104A3000BAF808301A06F7D402217F48A389FBF799
:104A4000DBFE20217C48FBF7D7FEEDB202217A483D
:104A5000FBF7D4FEA581B8F808309B07FBD0BAF865
:104A600008301806F7D402217348A389FBF7C4FE67
:104A700020217148FBF7C0FE02216F48FBF7BEFE04
:104A8000A4F80C90B8F808309907FBD0BAF80830B1
:104A90001A06F7D402216848A389FBF7ADFE20214E
:104AA0006548FBF7A9FE02216348FBF7A7FEA58135
:104AB000B8F808309B07FBD0BAF808301D06F7D4C9
:104AC00002215D48A389FBF797FE20215A48FBF796
:104AD00095FE02215848FBF791FE2B23A381B8F8DD
:104AE00008309807FBD0BAF808301906F7D402212D
:104AF0005148A389FBF780FE20214F48FBF77CFE3D
:104B00003D0A02214C48FBF779FEA581B8F8083030
:104B10009A07FBD0BAF808301B06F7D402214648A2
:104B2000A389FBF769FE20214348FBF765FEFFB22E
:104B300002214148FBF762FEA781B8F808309807C8
:104B4000FBD0BAF808301906F7D402213A48A389F5
:104B5000FBF752FE20213848FBF74EFE0221364873
:104B6000FBF74CFEA581B8F808309A07FBD0BAF8DD
:104B700008301B06F7D402212F48A389FBF73CFE1F
:104B800020212D48FBF738FE02212B48FBF736FE8B
:104B9000A781B8F808309D07FBD0BAF8083018068E
:104BA000F7D402212448A389FBF726FE20212248BE
:104BB000FBF724FE02212048FBF720FE2C23A381D3
:104BC000B8F808309907FBD0BAF808301A06F7D4BD
:104BD00002211948A389FBF70FFE20211648FBF795
:104BE0000BFE02211448FBF709FEBDF81030A3812B
:104BF000B8F808309B07FBD0BAF808301F06F7D486
:104C000002210D48A389FBF7F7FD20210A48FBF795
:104C1000F3FD02210848FBF7F1FD9DF84030A38128
:104C2000B8F808309D07FBD0BAF808301806F7D45A
:104C3000B4E601464CE500BF000C0240285F0020AE
:104C4000325F00202DE9F04782B0184F184DDDF893
:104C50002890DDF82C802980824614461E46388034
:104C6000227842B10A2A13D00D2A334606D10134E4
:104C70002278002AF6D102B0BDE8F087388829886A
:104C8000CDF80480CDF800900134FFF70BFDE7E785
:104C90002B887278013313442B8063780D2B06BF69
:104CA0000134002353463B800134D9E7285F0020BC
:104CB000325F00202DE9F04FBA4D8DB02C88029262
:104CC00084420793029BDDF858E09ABF04F1FF3657
:104CD000B6B206469C420F4602D8013CA3B20293EC
:104CE0006B88079ABB429CBF03F1FF37BFB2934268
:104CF00002D8013B9BB20793029A964280F0A481AE
:104D0000C6EB020B0FFA8BF30193079B9F42C0F097
:104D10009181C3EB07080FFA88F300934FF6FF73F6
:104D20000B9301230A93009B019A1946914280F24A
:104D30007A8102EBD2756D105FFA8EF30893CEF391
:104D400007230993330A0393F3B2DFF860B20593A4
:104D50003B0A0493FBB2D8465C4606932021924856
:104D6000FBF74CFD02219048FBF748FD2A23ABF8E6
:104D70000C30BBF808309A07FBD0B8F808301B0697
:104D8000F7D402218848A389FBF736FD2021864805
:104D9000FBF732FDBDF80CA083480221FBF72EFD86
:104DA000A4F80CA0BBF808309807FBD0B8F808307E
:104DB0001906F7D402217C48A389FBF71DFD2021A9
:104DC0007948FBF719FDBDF8149077480221FBF7ED
:104DD00015FDA4F80C90BBF808309A07FBD0B8F882
:104DE00008301B06F7D402216F48A389FBF704FDA6
:104DF00020216D48FBF700FD02216B48FBF7FEFC0C
:104E0000A4F80CA0BBF808309807FBD0B8F808301D
:104E10001906F7D402216448A389FBF7EDFC202191
:104E20006148FBF7E9FC02215F48FBF7E7FCA4F8C7
:104E30000C90BBF808309A07FBD0B8F808301B0676
:104E4000F7D402215848A389FBF7D6FC2021564805
:104E5000FBF7D4FC02215448FBF7D0FC2B23A381A1
:104E6000BBF808309807FBD0B8F808301906F7D41B
:104E700002214D48A389FBF7BFFC20214A48FBF7DC
:104E8000BBFCBDF810A048480221FBF7B7FCA4F812
:104E90000CA0BBF808309A07FBD0B8F808301B0606
:104EA000F7D402214048A389FBF7A6FC20213E4805
:104EB000FBF7A2FCBDF818903B480221FBF79EFCD3
:104EC000A4F80C90BBF808309807FBD0B8F808306D
:104ED0001906F7D402213448A389FBF78DFC202161
:104EE0003148FBF789FC02212F48FBF787FCA4F827
:104EF0000CA0BBF808309A07FBD0B8F808301B06A6
:104F0000F7D402212848A389FBF776FC2021264804
:104F1000FBF772FC02212448FBF770FCA4F80C900C
:104F2000BBF808309807FBD0B8F808301906F7D45A
:104F300002211D48A389FBF75FFC20211A48FBF7DB
:104F40005DFC02211848FBF759FC2C23A381BBF818
:104F500008309A07FBD0B8F808301B06F7D40221B6
:104F60001148A389FBF748FC20210F48FBF744FCBC
:104F700002210D48FBF742FCBDF82430A381BBF8A9
:104F800008309807FBD0B8F808301906F7D402218A
:104F90000548A389FBF730FC20210348FBF72CFCD4
:104FA000022105E02C5F0020000C0240003C004084
:104FB0003248FBF723FCBDF82030A381BBF8083052
:104FC0009A07FBD0B8F808301B06F7D402212B480B
:104FD000A389FBF711FC029B9E421ED0019B5B4202
:104FE0009D4218DD0A9B1E44B6B2009B320AEB1AA2
:104FF0000392F2B205921BB2009A954209DA0B9A1B
:105000001744019ABFB213443A0A0492FAB21BB28F
:1050100006921D46A2E62B46EEE7079B9F42DDD196
:105020000DB0BDE8F08F009B03EBD3756D106D42A2
:105030002DB281E6C7EB030801230FFA88F20B9328
:105040000A93009213466FE6C2EB060B079A0FFA1B
:105050008BF3974201930BD2C7EB02080FFA88F348
:10506000009301230B934FF6FF730A93009B5BE6BB
:10507000C2EB07084FF6FF73DFE700BF000C0240EA
:105080002DE9F04182B01D46089C009406468846F2
:105090000B461746FFF70EFE2B463246414630467A
:1050A0000094FFF707FE41462B463A4638460094E7
:1050B000FFF700FE3A4630462B462946089402B0D8
:1050C000BDE8F041FFF7F6BD2DE9F04182B099420D
:1050D000089E0ED20C461D468046174623462146A2
:1050E000013400963A464046A4B2FFF7E3FDA542DC
:1050F000F4D802B0BDE8F081704700BFF0B56B4B4B
:10510000984289B004460D4633D0694B98424FD03F
:10511000684B984201D009B0F0BD03AE3046FBF7B2
:10512000CFFB654A136C43F400431364002D00F079
:105130008380012D00F08B80032D59D000234FF088
:1051400082714FF000725B4C0391049306930592B9
:10515000238823F040031B041B0C23803146204688
:10516000FBF78EFB23889BB243F04003238009B0FA
:10517000F0BD03AE3046FBF7A3FB4F4A536C43F43C
:1051800080535364002D38D0012D6CD0032D03D1F2
:1051900020460521FFF7B0FF4FF0827000214FF04D
:1051A00000722023414C0390049105920693CFE7AF
:1051B00003AE3046FBF784FB3F4A136C43F4804355
:1051C00013642DB3012D64D0022D57D0032D03D1CC
:1051D00020460521FFF790FF4FF0827000214FF02D
:1051E00000722023324C0390049105920693AFE79E
:1051F00020460621FFF780FFA0E7032205238DE864
:105200000C00E0212B462A462C48FDF78BFBC3E718
:10521000032405272B462A468DE890004FF4806131
:105220002748FDF77FFB8DE890002B462A460C218E
:105230002448FDF777FBCFE7032206238DE80C0017
:1052400038212B462A461E48FDF76CFB76E70621DF
:1052500003220023019100924FF4E0511A461948AD
:10526000FDF760FB6AE7052103220023019100920C
:1052700038211A461248FDF755FB8DE70521032218
:105280000023019100920D211A460F48FDF74AFBB9
:10529000A2E7052103220023019100924FF460410F
:1052A0001A460748FDF73EFB96E700BF0030014075
:1052B00000380040003C004000380240000002403E
:1052C00000040240000802400020024008B52DED15
:1052D000048BB0EE409AF0EE608A00F013F8F0EE26
:1052E000680AB0EE408AB0EE490A00F011F8F0EE1C
:1052F000400AB0EE480ABDEC048BBDE8084000F05F
:105300000BB800BFB0EE600A82B002B0704700BFB9
:1053100082B002B0704700BF00F000B810B582B094
:10532000CDED010A019B23F00042B2F1FF4FF0EEF8
:10533000407A19DC10EE100A20F00041B1F1FF4F65
:1053400012DCB3F17E5F49D09C1704F0020444EAFA
:10535000D07479B9022C3ED09FED400A032C18BFBF
:10536000B0EE670A02B010BD9DED017A37EE270A54
:1053700002B010BD12B3B2F1FF4F34D0B1F1FF4F04
:105380001CD08A1AD2153C2A22DC002B4BDB9DED67
:10539000010A87EE800A00F053F900F075F8012C3D
:1053A0003AD0022C2FD0002CE2D09FED2D7ADFEDE9
:1053B0002D7A30EE070A30EE670AD9E7DFED2A7A58
:1053C0009FED2A0A0028A8BFB0EE670A02B010BD00
:1053D0009FED250AE3E79FED230AC9E702B0BDE888
:1053E000104000F051B8B1F1FF4F21D0022CF2D0A3
:1053F000032C2AD0DFED1E7A9FED1E0A012C08BF78
:10540000B0EE670AB4E79FED167ADFED167A30EE5C
:10541000070A37EEC00AABE710EE103A03F100437B
:1054200000EE103AA4E73C32B1DA9FED120AB6E77B
:10543000022C10D0032C0BD0DFED0F7A9FED0F0A5A
:10544000012C08BFB0EE670A92E79FED040A8FE7D0
:105450009FED0B0A8CE79FED0B0A89E7DB0F49C034
:105460002EBDBB33DB0F4940DB0FC93FDB0FC9BF8C
:105470000000008000000000DB0F49BFDB0F493F48
:10548000E4CB16C0E4CB164038B510EE105A25F028
:105490000044B4F1A14FF0EE407A0BDBB4F1FF4FC2
:1054A00058DCDFED547A9FED540A002DC8BFB0EEF2
:1054B000670A38BD514B9C425DDCB4F1445F4CDB64
:1054C0004FF0FF3367EEA75A9FED4D1A9FED4D2A1F
:1054D0009FED4D3ADFED4D1ADFED4D2A9FED4D4A20
:1054E000DFED4D3A9FED4D5ADFED4D4A9FED4D6A90
:1054F000DFED4D6A25EEA57A5A1CA7EE012AE7EEEC
:10550000212AA7EE023AE7EE223AA7EE034AE7EE97
:10551000234AA7EE045AE7EE246AA7EE056A26EEB0
:10552000877A66EE256A3ED0404A41499B001A447C
:1055300076EE876A92ED007A97EEA67A0B44002DFC
:1055400093ED000A77EE677A70EE677A28DBB0EEAB
:10555000670A38BD30EE000A38BD9FED367A30EE6E
:10556000077AF7EE006AB4EEE67AF1EE10FAA7DDFC
:10557000B0EE670A38BD00F063F82F4B9C4219DC8F
:10558000A3F5D0039C422ADCF0EE007ABFEE007A4D
:10559000A0EE277A002330EE270AC7EE007A91E7C3
:1055A000B1EE670A38BD76EE876AE7EEE67AB0EECE
:1055B000670A38BD214B9C420BDCF7EE087AB7EE48
:1055C000007AA0EE277A022330EE670AC0EE077A4F
:1055D00078E7BFEE007AC7EE007A032372E7F7EEB2
:1055E000007A30EE677A30EE270A0123C7EE007AA0
:1055F00068E700BFDB0FC93FDB0FC9BFFFFFDF3E1E
:10560000D769853C59DA4B3D356B883D21A215BDE4
:105610006BF16EBD6E2EBA3D95879DBD2549123E3C
:10562000388EE3BDABAAAA3ECDCC4CBE889D000807
:10563000989D0008CAF24971FFFF973FFFFF1B408A
:1056400010EE103A23F0004300EE103A704700BF0E
:1056500070B5960838D09FED257A01F1100400F15D
:105660000803354633F908EC07EE90EAF8EEE77ADE
:10567000013D67EE877A03F1080344ED047A33F9BC
:105680000EEC07EE90EAF8EEE77A04F1100467EE0C
:10569000877A44ED077A33F90CEC07EE90EAF8EEDE
:1056A000E77A67EE877A44ED067A33F90AEC07EE7B
:1056B00090EAF8EEE77A67EE877A44ED057AD1D181
:1056C00001EB061100EBC60012F003020DD09FEDB6
:1056D000077A30F9023B07EE903AF8EEE77A013AA2
:1056E00067EE877AE1EC017AF3D170BD00000038F3
:1056F000F0B497086ED0DFED495A00F1100501F1C2
:1057000008043E46B6EE006AFEEE006A55ED047AE5
:1057100027EEA57A1035B5EEC07AF1EE10FAD4BFB7
:10572000F0EE667AF0EE467A77EE877A0834FDEE90
:10573000E77A17EE903A03F30F0324F8103C55ED87
:10574000077A27EEA57AB5EEC07AF1EE10FAD4BF4B
:10575000F0EE667AF0EE467A77EE877AFDEEE77A3B
:1057600017EE903A03F30F0324F80E3C55ED067A3A
:1057700027EEA57AB5EEC07AF1EE10FAD4BFF0EEBE
:10578000667AF0EE467A77EE877AFDEEE77A17EEE4
:10579000903A03F30F0324F80C3C55ED057A27EEFD
:1057A000A57AB5EEC07AF1EE10FAD4BFF0EE667AC3
:1057B000F0EE467A77EE877A013EFDEEE77A17EE55
:1057C000903A03F30F0324F80A3C9FD100EB071033
:1057D00001EBC70112F003021ED0DFED105AB6EE46
:1057E000006AFEEE006AF0EC017A27EEA57AB5EECB
:1057F000C07AF1EE10FAD4BFF0EE667AF0EE467A97
:1058000077EE877A013AFDEEE77A17EE903A03F3E6
:105810000F0321F8023BE6D1F0BC704700000047BF
:105820002DE9F0414F1E5FEA970800F1040ED0ED1C
:10583000007A58D01430C4460426002410ED046ABF
:1058400050ED036A10ED027A50ED015AB4EEE76AAA
:10585000F1EE10FAC8BFF0EE467AA6F10305F4EEB9
:10586000E67AC8BF2C46F1EE10FA48BFF0EE667A31
:10587000A6F10205F4EEC77A48BF2C46F1EE10FA05
:1058800048BFF0EE477A06F1FF35F4EEE57A48BFFF
:105890002C46F1EE10FA48BF344648BFF0EE657A68
:1058A000BCF1010C06F1040600F11000C6D10EEBAC
:1058B000081E17F0030018D0081ABEEC017AB4EEE7
:1058C000E77AF1EE10FAC8BF044600F10100D8BF34
:1058D000B0EE677A8842F0EE477AEED182ED007A38
:1058E0001C60BDE8F0814446E3E7B0EE677AF5E777
:1058F0002DE9F0412DED088BB0F800E042684FEA49
:105900005E0C01EB8E085FEADE0E07464FEA8C0361
:1059100000F0AF801033CE181032434401F110056F
:1059200008F1100454ED041A13ED044A53ED033A40
:1059300053ED025A13ED015A54ED036A14ED020AB5
:1059400016ED042A56ED032A15ED036A15ED017ACA
:1059500015ED043A54ED017A56ED020A16ED011ADE
:1059600055ED024A73EE21BA36EE26BA37EE27AA73
:1059700072EE049A32EEA39A31EE058A74EE80AA92
:1059800070EEA58A45ED04BA05ED03BA45ED02AA0D
:1059900005ED01AA06ED018A46ED049A06ED039A8B
:1059A00046ED028A76EE666A73EEE23A12ED036A1B
:1059B00052ED042A33EE613A34EE424A26EE868AEC
:1059C00024EE062A63EE221A24EE224A23EE063A39
:1059D00066EEA26A23EE866A63EEA23A36EE046AA7
:1059E00076EEC36A72EE633A71EE882A44ED036A7A
:1059F00044ED042A43ED043A03ED036A77EE677A37
:105A000075EEE06A12ED017A52ED025A35EE416A06
:105A100074EEC04A67EE873A26EE875A24EEA54A0E
:105A200067EEA57A64EE874A66EEA56A26EE077AE7
:105A300026EE256A77EEE47A74EE235A35EE466A4E
:105A400037EE267ABEF1010E44ED025A05F110053B
:105A500044ED017A06F1100603ED026A03ED017AC6
:105A600002F1100204F1100403F110037FF45AAFA5
:105A70007A681FFA8CF408460223214601F040F8A8
:105A8000BDEC088B404621467A680223BDE8F04110
:105A900001F036B82DE9F04F2DED0A8B028891ED1B
:105AA000006A8FB00F46520893000C900391416832
:105AB00097ED017A38461844064609901844D0ED0F
:105AC000006AD6ED003AD6ED012AD0ED017A0A90AF
:105AD00076EE265A044625461C4494ED004A94ED81
:105AE000015A019475EEA34A304674EE244A3E46AC
:105AF00014EE90EA76EE666A46F808EB37EE276A0F
:105B0000D0ED014A049677EE677A019E32EEA63A0E
:105B100096ED012A36EE247A75EEE35A77EEE34AE3
:105B200036EE626A77EEA37A76EEE26A73EE453A73
:105B3000044636EE456A75EE266AA34637EE027ACB
:105B400034EE845A13EE908AA44675EEC45A87ED5B
:105B5000017A4BF8088BACF104078CED015A01F186
:105B6000080C2C46CDF814C015EE90CA44F808CBAA
:105B7000079401F1100485ED016A520802942C4645
:105B800001F118050B92B246069577EEC47A023AF7
:105B900016EE905AB646304652084AF8085BA0F115
:105BA0000406CEED017A089200F030819146039A06
:105BB000DDF80880CDF834A0083B02F1100501F1B2
:105BC000200CA4F10C0201F1300E33441034504685
:105BD000594655ED023A14ED025A91ED007AD0ED96
:105BE000007A15ED014A54ED015AD0ED016A91EDAC
:105BF000016A33EE858A34EE250A78EE074A74EEA0
:105C0000655A77EEA44A33EEC55A45ED024AD1ED06
:105C1000014A90ED014A70EE244A76EE05AA74EE30
:105C2000844A35EEC7AA45ED014AD6ED001AD7EDF4
:105C3000000A92ED024AD3ED023A93ED012A16EDE5
:105C4000011AD2ED012A57ED019A70EEA14A39EE00
:105C5000813A74EE848A70EEE11A73EEA88A7AEEC5
:105C6000E6AA18EE90AA47F808A9D2ED018A93EDAA
:105C7000019A73EE288A3AEE27AA78EE898A74EEA2
:105C8000630AC7ED018A18ED02BA58ED018A39EEB0
:105C9000C11A6AEE28BA2AEE8BCA71EEE29A30EE89
:105CA000819A79EE829A3CEE2BCA6AEEA8AA69EE36
:105CB000A8BA2AEE0BAA69EE8B9A69EE288A29EE19
:105CC0000BBA1CEE10AA78EEA98A41F808AB3AEE9E
:105CD0006AAA3BEECBBA34EEC44A33EE623A01ED27
:105CE00001AAC2ED018A82ED02BA5CED044A74EEAB
:105CF000633A38EE478A1CED034A30EE460A33EE2B
:105D0000423A38EE678A30EE660A23EEE49A63EE92
:105D1000048A28EE24AA60EE049A28EE048A20EE73
:105D2000240A63EE843A39EE684A7AEE299A14EE30
:105D300010AA30EE480A63EE244A44ED029A73EE4C
:105D4000E43A04ED010A46F808A935EE466A35EE54
:105D5000877AC6ED013A76EE866A77EE677A1EEDAF
:105D6000056A1EED067A67EE865A26EE875A72EEAF
:105D7000622A30EEC11A72EEE12A75EE255A62EE01
:105D8000860A66EE866A67EE877A21EE066A62EE1A
:105D9000872A21EE071A15EE90AA77EEE67A40F8E8
:105DA00008AB30EEC11A76EE222AB9F1010940EDB6
:105DB000017A05F1080583ED021AC3ED012A08F105
:105DC0000808A2F108020CF1100C04F108040EF10D
:105DD000180EA3F108037FF4FCAE08990298DDF8D1
:105DE00034A0CB0001EB410200EB011102910499B8
:105DF0001944049105991944059107999B44194444
:105E00009A44069B079103EBC2030693049A0798F2
:105E1000D2ED003A90ED004ADBED007A9AED003ABF
:105E2000D2ED014A90ED017A9BED012ADAED015A9B
:105E3000BDF82C400C9E73EE846A34EE876A36EE11
:105E4000A75A34EEC77A33EE055A33EEC44A82EDD0
:105E5000005A9BED015ADAED014A36EE055A72EE10
:105E6000043A35EE245A77EE674A82ED015A059AD4
:105E700034EE835AD2ED001AD2ED012A029A73EE63
:105E8000E53A36EE426A63EEA14A63EEA23A65EE67
:105E9000222A25EE215A74EEA22A35EE635A76EEB6
:105EA000E76ACBED002A8BED015AD2ED013A92ED73
:105EB000005A069A76EEC36A36EE656A66EE854A41
:105EC00026EE055A66EEA36A26EE236A75EE666A2A
:105ED00034EE866A34EE424A37EE277AC0ED016A24
:105EE00080ED006A92ED016A039877EE437A75EED1
:105EF000845A92ED007A65EE876A27EE877A65EE1E
:105F0000865A67EE867A77EE655A76EEA77ACAEDFC
:105F1000015ACAED007A72682146042300F0F0FDB0
:105F2000099872682146042300F0EAFD0A98726815
:105F30002146042300F0E4FD019872682146042301
:105F40000FB0BDEC0A8BBDE8F04F00F0D9BD00BF2B
:105F50002DE9F041012A064617460C469846058869
:105F600054D0B5F5807F4CD016D9B5F5806F1AD0D6
:105F70005CD9B5F5006F44D0B5F5805F05D12046FA
:105F800029467268012300F0BBFDB8F1000F11D162
:105F9000012F16D0BDE8F081202D32D04AD9402DF6
:105FA000EDD0802DF1D130462146FFF7A1FCB8F1AC
:105FB000000FEDD02046B189B26800F041FD012FFD
:105FC000E8D107EE905AF8EE676AF7EE007AC7EE6E
:105FD000A66A002DDED004F10801002301339D42A2
:105FE00001F1080111ED047A51ED037A27EE267ACA
:105FF00067EEE67A01ED047A41ED037AEED1BDE871
:10600000F08130462146FFF745FDBEE7ADB101F115
:106010000C03002253ED027A0132F1EE677A9542C9
:1060200043ED027A03F10803F4D19AE7B5F5007F56
:10603000A5D0AAE7102DB6D0A7E7B5F5807F94D8F4
:10604000AAE700BF70B52DED028B069C826004F1BB
:106050008044013C05460C44B0EE408A01801E4657
:10606000A2001846002101F0A7FD6E6085ED038AAD
:10607000BDEC028B70BD00BF2DE9F04F85B0054629
:106080000290008801900446D5F80480D5F808A055
:1060900095ED033A04F18040013808EB80090F9830
:1060A000002800F0E780A6088446300108EB000EC7
:1060B00045465044CDF80C80DDF83880009004F05F
:1060C000030751F8040B49F8040B9FED6B7A002E7F
:1060D00000F0CD8005F110040AF11000B34654ED34
:1060E000043A50ED047A14ED036A50ED034A14EDBE
:1060F000024A50ED025A14ED015A50ED016A63EE66
:10610000A77A66EE244A77EE877A64EE255A34EE53
:10611000A76A65EE266A35EE867ABBF1010B04F1BB
:10612000100436EE877A00F11000D8D1DDF800B007
:10613000744657B13846F4EC016AFBEC017A66EE1E
:10614000A77A013837EE277AF5D1A3EC017AF2EC81
:10615000017A77EEC77AE8EC017A67EE837A002E4F
:1061600000F0828005F110040AF11000B34614ED2E
:10617000047A10ED045A50ED035A10ED026A50ED06
:10618000016A27EE877ABBF1010B35EE077A04F13D
:10619000100400ED047A14ED077A27EE877A00F1F7
:1061A000100035EE877A00ED077A14ED067A27EEB7
:1061B000877A36EE077A00ED067A14ED057A27EE37
:1061C000877A36EE877A00ED057AD0D10098F346CB
:1061D0003C465FB1BBEC017AD0ED006A27EE877ACE
:1061E000013C36EE877AA0EC017AF3D1BCF1010CC8
:1061F00005F104050EF1040E7FF463AF0F9BDDF88B
:106200000C8008EB8308029B5C68019B591E8E087A
:106210001DD004F1100208F11003304653F8105C51
:1062200042F8105C53F80C5C42F80C5C53F8085CC4
:1062300042F8085C53F8045C42F8045C013803F14E
:10624000100302F11002E9D133011C44984411F00B
:10625000030306D0224658F8041B42F8041B013BF6
:10626000F9D105B0BDE8F08F5046AB46B0E7D34654
:106270002C465EE74446C8E70000000070B5049C69
:10628000826004F18044013C05460C4401801E46B6
:10629000A2001846002101F08FFC6E6070BD00BFA7
:1062A0002DE9F04F2DED108B89B005460390008845
:1062B000D5F804C004931E4600F18043013B0CEB6B
:1062C0008304F308D5F808800190254600940293D2
:1062D00000F0EE814FEAD0099E464FEA49131E1F97
:1062E0000446059608EB030004F0070A13460CF178
:1062F0002004CDF818C084464846DDF81490079174
:1063000005F1200701F1200602F1200552469A46C8
:1063100056F8203C47F8203C56F81C3C47F81C3CFB
:1063200056F8183C47F8183C56F8143C47F8143C0B
:1063300056F8103C47F8103C56F80C3C47F80C3C1B
:1063400056F8083C47F8083CDFEDF13A56F8043CB3
:1063500047F8043C14ED083A54ED072A14ED062AD8
:1063600054ED051A14ED041A54ED030A14ED020A53
:10637000211FF0EE638AF0EE639AF0EE63AAF0EE6E
:1063800063BAB0EE63CAF0EE63CAB0EE63DA002817
:1063900000F0E88108F1200104F11C03834613EDAD
:1063A000088A11ED084A51ED074A11ED065A51EDE0
:1063B000055A11ED046A51ED036A11ED027A51EDAF
:1063C000017A23EE04FA62EE84EA13ED073A22EE34
:1063D00004EA61EE84DA21EE04BA20EE84AA20EE0B
:1063E000049A28EE044A62EE24FA3CEE0ECA7BEED2
:1063F000ADBA21EEA4EA61EE24DA7AEE8BAA79EE48
:106400008A9A20EEA4BA20EE24AA3DEE0FDA7CEEA2
:10641000AECA22EEA4FA78EE898A53ED062A28EE57
:10642000249A73EE843A63EE244A22EE054A61EE22
:1064300005EA13ED052A3DEE0FDA7CEEAFCA20EE39
:1064400085FA61EE85FA3CEE0EEA7BEEADDA3AEEC5
:106450008BBA60EE05BA68EE05AA39EE8AAA78EE24
:10646000898A73EEA43A63EE054A22EE855A21EE3C
:10647000259A20EE25CA3DEE04DA7CEEAFCA21EE65
:10648000A54A3EEE2EEA53ED041A60EEA5EA7DEE33
:106490008FDA3BEE2BBA3AEE2AAA68EE25BA63EE03
:1064A00025AA78EEA48A73EE853A22EEA55A62EE0A
:1064B000255A61EE064A60EE869A60EE06FA13ED02
:1064C000031A23EE06FA3DEE04DA7CEE89CA3EEEAC
:1064D0002EEA28EE069A7DEE8CDA3BEE2BBA22EEFF
:1064E00086CA3AEE2AAA78EE858A73EEA53A62EE5B
:1064F000065A21EE866A20EE264A63EE26EA3AEE36
:106500000CAA22EE265A3DEE24DA7CEEA9CA60EEF1
:10651000A64A3EEE2FEA53ED020A68EE26FA7DEE19
:1065200089DA3BEE0FBA78EEA58A22EEA6FA73EE70
:10653000863A21EEA66A61EE266A60EE07AA28EE88
:1065400007CA63EE07BA7AEE059A78EE868A3DEEC0
:1065500024DA7CEE84CA7DEEAEDA22EE079A62EE91
:1065600087EA61EE875A73EEA63A13ED010A61EEEF
:10657000076A3EEE2FEA3BEE0FBA20EE877A68EE0E
:10658000274A3DEE2ADA7CEE8CCA23EE278A3EEEBD
:106590002BEA22EEA74A22EE27AA21EEA75A21EEE5
:1065A000276A78EEA66A7DEEAEDA60EEA78A3BEE49
:1065B00009BA79EEA59A73EE873A60EE277ABBF1B5
:1065C000010B01F120013DEE24DA7CEE88CA3EEE9B
:1065D00004CA7DEE8ABA7BEE05AA79EE869A76EE3B
:1065E000A88A73EEA73A03F120037FF4D8AE09EB33
:1065F0000401E346A2B31346BBEC016AF1EC017A55
:1066000023EE063A22EE864A62EE064A21EE865ACA
:1066100061EE065A60EE866A20EE067A27EE866AFA
:10662000013B3DEE03DA7CEE84CAB0EE623A3CEE0A
:1066300024CAF0EE422A7BEE85BAB0EE612A7AEEE9
:10664000A5AAF0EE411A79EEA69AB0EE601A78EE9D
:10665000878AF0EE400A73EE863AB0EE670ACBD135
:10666000BEF1010E05ED08DA45ED07CA05ED06CAD3
:1066700045ED05BA45ED04AA45ED039A45ED028ABC
:1066800045ED013A07F1200706F1200604F1200448
:1066900005F120057FF43CAE029B0098DDF818C0A0
:1066A00007995B0152461844009019449C441A44CF
:1066B000049B13F0070E1FD0009FDDF80490764670
:1066C000654651F8043BDFED126A47F8043B444647
:1066D0004B462846B0EC017AF4EC017A67EE277A53
:1066E000013B76EEA76AF5D1013EE2EC016A05F1C5
:1066F0000405E6D10CEB8E0C019B591E039B8E0802
:106700005C6820D004F110020CF11003304601E067
:106710000000000053F8105C42F8105C53F80C5C69
:1067200042F80C5C53F8085C42F8085C53F8045CCF
:1067300042F8045C013803F1100302F11002E9D1C0
:1067400033011C449C4411F0030306D022465CF83C
:10675000041B42F8041B013BF9D109B0BDEC108BBE
:10676000BDE8F08FC34645E72DE9F0415FEA9208A6
:1067700084B07FD0002700F1200401F110054646C7
:106780005AE0B1EEE70AB4EE400AF1EE10FA40F03A
:10679000A48005ED040A54ED067A14ED050A67EEAF
:1067A000A77A20EE000A77EE807AF5EEC07AF1EE55
:1067B00010FAC0F28F80B1EEE70AB4EE400AF1EEB3
:1067C00010FA40F0AF8005ED030A54ED047A14EDA1
:1067D000030A67EEA77A20EE000A77EE807AF5EEDC
:1067E000C07AF1EE10FA72DBB1EEE70AB4EE400ABD
:1067F000F1EE10FA40F08C8005ED020A54ED027AB9
:1068000014ED010A67EEA77A20EE000A77EE807A8F
:10681000F5EEC07AF1EE10FA20DBB1EEE70AB4EE45
:10682000400AF1EE10FA69D1013E05ED010A04F1CA
:10683000200405F1100519D054ED087A14ED070A6B
:1068400067EEA77A20EE000A77EE807AF5EEC07A3E
:10685000F1EE10FA95DA45F8107C9CE7013E45F818
:10686000047C04F1200405F11005E5D100EB48108B
:1068700001EB081112F0030526D0002600F10804F0
:106880000CE0B1EEE70AB4EE400AF1EE10FA2ED1B8
:10689000013D01ED010A04F1080415D054ED027A1E
:1068A00014ED010A67EEA77A20EE000A043177EEB4
:1068B000807AF5EEC07AF1EE10FAE2DA013D41F8A5
:1068C000046C04F10804E9D104B0BDE8F08145F896
:1068D000087C93E745F80C7C77E7B0EE670A0392F3
:1068E0000291019000F0EEFB01A807C851E7B0EE5D
:1068F000670A019100F0E6FB0199C9E7B0EE670A6B
:1069000003920291019000F0DDFB01A807C88BE71C
:10691000B0EE670A03920291019000F0D3FB01A848
:1069200007C869E7B0EE670A03920291019000F090
:10693000C9FB01A807C846E79FED1E7AB5EEC00A5D
:1069400020EE077AF1EE10FAFDEEC77A2CD4F8EEBD
:10695000E77ADFED196A194A77EE677AB7EE000A2F
:1069600067EEA67AF4EEE67AF1EE10FAA8BF77EEBB
:10697000E67ABCEEE77A17EE103AC3F3080307EEA7
:10698000103AB8EE477A02EB830177EEC77AD1ED81
:10699000016A30EE677A91ED000A67EEA67A27EE7B
:1069A000000A30EE270A704717EE903A013B07EED7
:1069B000903ACCE783F9223E00000044B8A50008D5
:1069C000DFED1C7A20EE270AF5EE007A30EE270A7A
:1069D000B5EEC00AF1EE10FAFDEEC07A04D517EE5E
:1069E000903A013B07EE903AF8EEE77ADFED126A53
:1069F000124A30EE670AB7EE007A20EE260AFCEE65
:106A0000C07A17EE903AC3F3080307EE903AF8EE17
:106A1000677A02EB830170EE677AD1ED016A91ED3E
:106A2000000A37EE677A67EEA67A27EE000A30EEA4
:106A3000270A704783F9223E00000044B8A50008E9
:106A40004B1C012B98BF70472DE9F003911C9B084C
:106A5000B1F80480B1F802900A8831F802CC804481
:106A6000814402448444D9F80070D8F80060156865
:106A7000DCF80040C9F80060C8F80070CCF800509D
:106A80001460D9F80470D8F804605568DCF8044044
:106A9000C9F80460C8F80470CCF804505460083198
:106AA000013BD5D1BDE8F00370474B1C012B98BFCB
:106AB00070472DE9F003911C9B08B1F80480B1F8F0
:106AC00002900A8831F802CC00EB580800EB590913
:106AD00000EB520200EB5C0CD9F80070D8F80060B3
:106AE0001568DCF80040C9F80060C8F80070CCF800
:106AF000005014600831013BDFD1BDE8F00370475E
:106B00002DE9F04F2DED108B9DB01C469FEDC8BABE
:106B10001A92031D824689468B461B9300949E461B
:106B20004FEADB035A00D618F51803925A19D01809
:106B3000DF0019183C46019757440C930AEBC20238
:106B40001B010AEBC10107EB040C009C02930AEB4A
:106B5000C6060AEBC505043204310AEBC0004FEA51
:106B6000CB034FF00008DCED007AD7ED006AD6EDDC
:106B7000003A5EED01AAD5ED004A90ED002A12ED33
:106B8000017A51ED010A77EE828A33EEA04A76EE61
:106B9000871A3AEEA43A31EE846A33EE285A36EE7A
:106BA000C77A75EE066A35EE465A4EED016A85EDF6
:106BB000005A96ED011AD7ED015A92ED00AA91ED17
:106BC000006A9EED009A95ED015ADCED016AD0ED68
:106BD000019A73EEE00A71EE462A75EECA3A37EE74
:106BE000600A33EEA28A37EE207A73EEE22A37EE9D
:106BF000C22A79EE053A60EE0B0A39EE455A7AEE72
:106C0000E44A36EEA99A75EE8A5A31EE066A76EEB5
:106C1000E96A28EE0B8A62EE8B2A67EE0B7A33EE76
:106C2000683A36EE880A75EE868A36EEC87A71EED4
:106C3000C41A75EE626A33EEC94A35EEC66A33EE9F
:106C4000891A74EEE05A74EEA03A75EE224A32EEDA
:106C5000275A72EE677A33EE068A75EE872A31EE8E
:106C6000289A33EE466A74EE610A33EE802A35EED6
:106C7000C77A34EEC53A76EEE75A31EE681A34EE4A
:106C8000214A73EEC03A74EE854A76EEA76AD8447C
:106C9000C1458EED009A85ED011A9E448CED008A67
:106CA0001D4480ED006ACCED010A80ED014A9C4450
:106CB00087ED002A184441ED013A42ED012A86EDA4
:106CC000007A87ED013AC1ED004A1F44C2ED005A37
:106CD0001944C6ED016A1A441E443FF644AF0C99AC
:106CE0000729204640F2E98104EB44073E19351993
:106CF000039C00902246013202EB81020099281881
:106D000000EB010E0C990A4404EB010C4FEACE048F
:106D10000AEBC20E009A0F94ED001195D5000D9567
:106D2000019D08351695029D0835140117950F9A97
:106D30001A9D0E94C0001090AA180792109A0C9CED
:106D4000AA180892119AAA18099201EB81010EF172
:106D500004020A92C9000D9A0C31F6004FEACC00E9
:106D60001491A9180E9A1296FF00AE1908304FEA36
:106D70000C1C06961990AA186401EE190CF10C006F
:106D80001397049615900391059204F10802189246
:106D90004FF00108002202F108010F460B911899EB
:106DA0008E1816998D1817998C1819998818149996
:106DB00001EB020C15990A440399D1ED00FA0599EB
:106DC00091ED00FA0499D1ED00EA069991ED00EAFF
:106DD0000999D1ED00DA089991ED00DA0799D1ED22
:106DE00000CA039991ED01CA0599D1ED01BA049940
:106DF000D1ED01AA069991ED01AA0999D1ED017A87
:106E00000899CDED007AD1ED017A0799CDED017A9F
:106E1000D1ED017A0AEB070E0A9FCDED027A0CEB59
:106E20000A0156445544544450445244C44601E077
:106E3000F304353F96ED005A52ED019A11ED016AC7
:106E4000D0ED007A17ED017ADEED003A94ED003ACC
:106E500095ED002A9EED010A33EE858A32EE061A80
:106E600033EE294A77EE874A78EE041A71EE246AE7
:106E700032EE462A31EEA66A77EEC77A8EED006AC8
:106E8000D0ED018A95ED019AD1ED002A97ED007AB7
:106E9000D4ED010A96ED016AD2ED005A73EEC53ABF
:106EA00033EE693A39EE625A78EEC79A38EE444AC0
:106EB00038EE877A30EEA58A79EE222A75EE698A55
:106EC00032EE279A35EE295A72EE677A30EE062AAC
:106ED00069EE0B9A70EEE55A32EE089A68EE8B8AEC
:106EE00032EE482A71EE644A25EE0B5A32EE871ACA
:106EF00067EE8B7A72EEC72A30EE466A73EE290A85
:106F000036EE280A33EE693A32EE647A73EEA79AC7
:106F100036EE686A73EEE77A75EE858A74EE223A89
:106F200035EEC55A71EEE66A79EE411A39EEA88A55
:106F300076EE435A74EE622A72EE244A30EE604ACC
:106F400079EEE88A30EE200A77EE859A36EE036A0B
:106F500077EEC57A2EEE212A2EEE265A6FEE230A00
:106F60002AEE213A39EE011A6AEE266A2BEE879A4A
:106F70006BEEA33A2FEE077A6FEE841A35EE033AE2
:106F800072EE666A2CEE045A2FEE882A9DED024AB4
:106F90008EED011A77EE633A2CEE088A9DED017AA8
:106FA00086ED003A30EE899A32EE052A6DEE220A1D
:106FB00031EEC88A67EE222A64EE001A27EE247AA0
:106FC0002CEEA85A6DEE244A64EE288A9DED004A04
:106FD000C6ED016A74EEE22A6DEEA94A64EE299AC2
:106FE00024EE254A30EE877A74EE844A6EEEA70AC4
:106FF0002AEE864A2CEE800A6DEEA55A6AEEA77A32
:107000002EEE866A75EE211A30EE680A75EEE99A60
:1070100070EE840A36EE676ADC44E14584ED009A3E
:10702000C4ED013A9E4402ED017AC2ED002A1E44ED
:1070300085ED002A85ED018A1C4447ED011A87ED94
:10704000000A1A4441ED014AC1ED009A1D44C0ED09
:10705000000A1F4480ED016A194418443FF6EAAE65
:10706000039A0D990A4403920E99059A0A440592CF
:107070001399049A0A4404921299069A0A440692B1
:107080001199099A0A4409921099089A0A44089297
:107090000F99079A0A4407920C990A9A08F1010875
:1070A000083288450A920B9A7FF475AEBDF83430E9
:1070B0000093C346DDF86CE032E51DB0BDEC108BEB
:1070C000BDE8F08F10B52DED028B8AB0B0EE408A8E
:1070D00000F04EF8244B93F90040631C09D0B4EE45
:1070E000488AF1EE10FA04D6B5EEC08AF1EE10FA35
:1070F00003D40AB0BDEC028B10BD01231B4A0093E0
:1071000018EE100A00230192089300F05FFA0022A3
:10711000CDE90401CDE902010023BCB110461946B6
:1071200000F0D2FB022CCDE9060111D100F004FDE4
:1071300021230360089B8BB9DDE9060100F0ACFC5C
:1071400000EE100A0AB0BDEC028B10BDCDE906239B
:10715000684600F05FF80028ECD1E7E700F0ECFCAF
:10716000089B0360E8E700BF900100202CB10008F5
:1071700010EE103A23F00042B2F1FF4F70B430D25B
:107180006AB3002B3DDBB2F5000F4FEAE3502CD37E
:10719000A0F17F02C3F31603D10743F4000348BFF5
:1071A0005B00002456105B00254619214FF08072C9
:1071B000A818984202DC1B1A8518144401394FEABA
:1071C00043034FEA5202F3D113B104F001031C440C
:1071D000641004F17C5404EBC65300EE103A70BC0A
:1071E0007047A0EE000A70BC704713F4000201D093
:1071F0000CE00A465B001C0202F10101F9D5801A7D
:10720000C6E770EE407A87EEA70AE8E74FF0FF3254
:10721000F5E700BF002070472DE9FF47DFF89890A1
:10722000CDF804904FF003080023CDF80C80012422
:10723000029301AF20463946ABBE05461A4ECDF843
:1072400004900423CDF80C80356002932046394623
:10725000ABBE8246154DCDF804900823CDF80C80C6
:10726000C5F800A0029320463946ABBE0446104A3A
:1072700010481460013404BF2B68136000214FF0E4
:10728000FF3440F83140013114290A4BF9D13168FB
:10729000286812681960002159609860D9601A61E5
:1072A000596104B0BDE8F087242100201C21002092
:1072B000282100202C21002034B100080D4B1A6831
:1072C00010B50AB90C4A1A601A6869461044884217
:1072D00006D80A490A4C0968A14208D0884206D952
:1072E00000F02AFC0C2303604FF0FF3010BD186043
:1072F000104610BD20210020385F0020940100209E
:10730000ADDEFECA81F0004102E000BF83F0004321
:1073100030B54FEA41044FEA430594EA050F08BF30
:1073200090EA020F1FBF54EA000C55EA020C7FEAF4
:10733000645C7FEA655C00F0E2804FEA5454D4EB71
:107340005555B8BF6D420CDD2C4480EA020281EA3B
:10735000030382EA000083EA010180EA020281EA73
:107360000303362D88BF30BD11F0004F4FEA0131C5
:107370004FF4801C4CEA113102D0404261EB4101D4
:1073800013F0004F4FEA03334CEA133302D052425A
:1073900063EB430394EA050F00F0A780A4F1010416
:1073A000D5F1200E0DDB02FA0EFC22FA05F2801850
:1073B00041F1000103FA0EF2801843FA05F3594136
:1073C0000EE0A5F120050EF1200E012A03FA0EFCB5
:1073D00028BF4CF0020C43FA05F3C01851EBE371DF
:1073E00001F0004507D54FF0000EDCF1000C7EEBFC
:1073F00000006EEB0101B1F5801F1BD3B1F5001F3A
:107400000CD349085FEA30004FEA3C0C04F1010458
:107410004FEA445212F5800F80F09A80BCF1004F81
:1074200008BF5FEA500C50F1000041EB045141EA03
:10743000050130BD5FEA4C0C404141EB010111F404
:10744000801FA4F10104E9D191F0000F04BF0146AF
:107450000020B1FA81F308BF2033A3F10B03B3F18D
:1074600020020CDA0C3208DD02F1140CC2F10C021D
:1074700001FA0CF021FA02F10CE002F11402D8BF7B
:10748000C2F1200C01FA02F120FA0CFCDCBF41EA47
:107490000C019040E41AA2BF01EB0451294330BD16
:1074A0006FEA04041F3C1CDA0C340EDC04F11404F3
:1074B000C4F1200220FA04F001FA02F340EA0300CA
:1074C00021FA04F345EA030130BDC4F10C04C4F110
:1074D000200220FA02F001FA04F340EA03002946F0
:1074E00030BD21FA04F0294630BD94F0000F83F43A
:1074F000801306BF81F480110134013D4EE77FEA1D
:10750000645C18BF7FEA655C29D094EA050F08BF68
:1075100090EA020F05D054EA000C04BF1946104649
:1075200030BD91EA030F1EBF0021002030BD5FEA8D
:10753000545C05D14000494128BF41F0004130BDB5
:1075400014F580043CBF01F5801130BD01F0004509
:1075500045F0FE4141F470014FF0000030BD7FEA7C
:10756000645C1ABF194610467FEA655C1CBF0B4677
:10757000024650EA013406BF52EA033591EA030F8E
:1075800041F4002130BD00BF90F0000F04BF002186
:10759000704730B54FF4806404F132044FF00005B9
:1075A0004FF0000150E700BF90F0000F04BF002132
:1075B000704730B54FF4806404F1320410F0004598
:1075C00048BF40424FF000013EE700BF42004FEA93
:1075D000E2014FEA31014FEA02701FBF12F07F4310
:1075E00093F07F4F81F06051704792F0000F14BF0D
:1075F00093F07F4F704730B54FF4607401F0004551
:1076000021F0004120E700BF50EA010208BF7047A7
:1076100030B54FF000050AE050EA010208BF70479C
:1076200030B511F0004502D5404261EB41014FF405
:10763000806404F132045FEA915C3FF4DCAE4FF009
:1076400003025FEADC0C18BF03325FEADC0C18BFF0
:10765000033202EBDC02C2F1200300FA03FC20FA41
:1076600002F001FA03FE40EA0E0021FA02F114448E
:10767000C1E600BF70B54FF0FF0C4CF4E06C1CEAA3
:1076800011541DBF1CEA135594EA0C0F95EA0C0F18
:1076900000F0DEF82C4481EA030621EA4C5123EA8B
:1076A0004C5350EA013518BF52EA033541F48011BA
:1076B00043F4801338D0A0FB02CE4FF00005E1FB6D
:1076C00002E506F00042E0FB03E54FF00006E1FBB7
:1076D00003569CF0000F18BF4EF0010EA4F1FF04FA
:1076E000B6F5007F64F5407404D25FEA4E0E6D413A
:1076F00046EB060642EAC62141EA55514FEAC5204B
:1077000040EA5E504FEACE2EB4F1FD0C88BFBCF5C6
:10771000E06F1ED8BEF1004F08BF5FEA500E50F177
:10772000000041EB045170BD06F0004646EA01013D
:1077300040EA020081EA0301B4EB5C04C2BFD4EB6F
:107740000C0541EA045170BD41F480114FF0000E68
:10775000013C00F3AB8014F1360FDEBF002001F0D6
:10776000004170BDC4F10004203C35DA0C341BDC50
:1077700004F11404C4F1200500FA05F320FA04F022
:1077800001FA05F240EA020001F0004221F0004156
:1077900010EBD37021FA04F642EB06015EEA430EC9
:1077A00008BF20EAD37070BDC4F10C04C4F12005F9
:1077B00000FA04F320FA05F001FA04F240EA0200AC
:1077C00001F0004110EBD37041F100015EEA430E7D
:1077D00008BF20EAD37070BDC4F1200500FA05F29D
:1077E0004EEA020E20FA04F301FA05F243EA02031C
:1077F00021FA04F001F0004121FA04F220EA02002B
:1078000000EBD3705EEA430E08BF20EAD37070BD70
:1078100094F0000F0FD101F00046400041EB010150
:1078200011F4801F08BF013CF7D041EA060195F032
:10783000000F18BF704703F00046520043EB0303EC
:1078400013F4801F08BF013DF7D043EA06037047D9
:1078500094EA0C0F0CEA135518BF95EA0C0F0CD0E4
:1078600050EA410618BF52EA4306D1D181EA03012A
:1078700001F000414FF0000070BD50EA410606BF24
:107880001046194652EA430619D094EA0C0F02D169
:1078900050EA013613D195EA0C0F05D152EA0336AE
:1078A0001CBF104619460AD181EA030101F00041CC
:1078B00041F0FE4141F470014FF0000070BD41F015
:1078C000FE4141F4780170BD70B54FF0FF0C4CF4EF
:1078D000E06C1CEA11541DBF1CEA135594EA0C0F0E
:1078E00095EA0C0F00F0A7F8A4EB050481EA030E5B
:1078F00052EA03354FEA013100F088804FEA033342
:107900004FF0805545EA131343EA12634FEA02220F
:1079100045EA111545EA10654FEA00260EF00041D0
:107920009D4208BF964244F1FD0404F5407402D222
:107930005B084FEA3202B61A65EB03055B084FEAB3
:1079400032024FF480104FF4002CB6EB020E75EBB0
:10795000030E22BFB61A754640EA0C005B084FEAD8
:107960003202B6EB020E75EB030E22BFB61A754655
:1079700040EA5C005B084FEA3202B6EB020E75EBA0
:10798000030E22BFB61A754640EA9C005B084FEA18
:107990003202B6EB020E75EB030E22BFB61A754625
:1079A00040EADC0055EA060E18D04FEA051545EA14
:1079B00016754FEA06164FEAC30343EA52734FEABD
:1079C000C2025FEA1C1CC0D111F4801F0BD141EA36
:1079D00000014FF000004FF0004CB6E711F4801F9B
:1079E00004BF01430020B4F1FD0C88BFBCF5E06F7B
:1079F0003FF6AFAEB5EB030C04BFB6EB020C5FEA8B
:107A0000500C50F1000041EB045170BD0EF0004EDF
:107A10004EEA113114EB5C04C2BFD4EB0C0541EA11
:107A2000045170BD41F480114FF0000E013C90E60E
:107A300045EA060E8DE60CEA135594EA0C0F08BFD2
:107A400095EA0C0F3FF43BAF94EA0C0F0AD150EAD1
:107A500001347FF434AF95EA0C0F7FF425AF104664
:107A600019462CE795EA0C0F06D152EA03353FF48C
:107A7000FDAE1046194622E750EA410618BF52EA09
:107A800043067FF4C5AE50EA41047FF40DAF52EADD
:107A900043057FF4EBAE12E74FEA4102B2F1E04357
:107AA00024BFB3F5001CDCF1FE5C0DD901F0004CE5
:107AB0004FEAC0024CEA5070B2F1004F40EB830035
:107AC00008BF20F00100704711F0804F21D113F161
:107AD0003872BCBF01F00040704741F480114FEA9A
:107AE0005252C2F11802C2F1200C10FA0CF320FA23
:107AF00002F018BF40F001004FEAC1234FEAD32340
:107B000003FA0CFC40EA0C0023FA02F34FEA4303A9
:107B1000CCE77FEA625307D150EA01331EBF4FF032
:107B2000FE4040F44000704701F0004040F0FE404D
:107B300040F40000704700BF014B1868704700BF59
:107B4000F801002008B5074B044613B10021AFF33C
:107B50000080054B1868836A03B19847204600F0FF
:107B6000A5FC00BF000000009CB1000870B50E4BE2
:107B70000E4CE41AA41000251E46A54204D056F867
:107B8000253098470135F8E700F0A4FC084C094B74
:107B9000E41AA41000251E46A54204D056F825304C
:107BA00098470135F8E770BDFC010020FC0100207A
:107BB00000020020FC01002002440346934202D050
:107BC00003F8011BFAE7704770B5CD1C25F00305DB
:107BD00008350C2D38BF0C25002D064601DBA942C7
:107BE00002D90C23336046E000F080F8234B1C6878
:107BF0001A462146A1B10B685B1B0ED40B2B03D98F
:107C00000B60CC18CD501EE08C420DBF63684B68F2
:107C10006360136018BF0C4615E00C464968E9E73D
:107C2000174C23681BB9304600F02CF82060294619
:107C3000304600F027F8431C18D0C41C24F003047D
:107C4000A0420DD12560304600F051F804F10B0040
:107C5000231D20F00700C31A0ED05A42E25070BD17
:107C6000211A304600F00EF80130EBD10C233360BE
:107C7000304600F03CF8002070BD00BFD02100204D
:107C8000CC21002038B5064C002305460846236069
:107C9000FFF714FB431C02D1236803B12B6038BDEE
:107CA000345F00200EB400B59CB04FF402711DABE0
:107CB000ADF81410029006906FF000410A4804914C
:107CC00007914FF6FF7153F8042BADF816100068BA
:107CD000019302A900F0B4F8029B00221A701CB0B4
:107CE0005DF804EB03B07047F8010020704770475F
:107CF00038B50546002946D051F8043C0C1F002B2E
:107D0000B8BFE418FFF7F2FF1F4A1368114613B912
:107D10006360146032E0A3420ED92268A018834247
:107D200004BF18685B68636004BF121822600C60AF
:107D300024E0A24203D813465A68002AF9D11868F1
:107D40001918A1420BD121680144581882421960C8
:107D500014D1106852685A60014419600EE002D9CB
:107D60000C232B600AE021686018824204BF10686F
:107D70005268626004BF091821605C602846BDE853
:107D80003840FFF7B4BF38BDD02100202DE9F047BF
:107D90008E689E4282460C46914698463ED88A8915
:107DA00012F4906F3AD0256809696F1A6569022349
:107DB00005EB450595FBF3F57B1C43449D4238BF1D
:107DC0001D4653050FD52946FFF7FEFE064698B11E
:107DD0003A46216900F014FBA38923F4906343F031
:107DE0008003A38113E02A4600F030FB064670B9F9
:107DF00021695046FFF77CFF0C23CAF80030A389A5
:107E000043F04003A3814FF0FF30BDE8F0872661C7
:107E100065613E44ED1B2660A5604646464528BF89
:107E2000464632464946206800F0F5FAA3689B1B97
:107E3000A36023681E4426600020BDE8F087000090
:107E40002DE9F04F9DB0804603938B891C060D46AB
:107E500016460DD50B695BB94021FFF7B5FE2860CA
:107E6000286118B90C23C8F80030CDE040236B61BD
:107E70000023099320238DF82930DFF89CB13023AB
:107E80008DF82A3037463C4614F8013B1BB9B7EB56
:107E9000060910D003E0252BF9D02746F3E74B461F
:107EA000324629464046FFF771FF013000F0A780B7
:107EB000099B4B4409933B78002B00F0A0800023E2
:107EC0004FF0FF3204930793059206938DF85330D9
:107ED0001A930126052221784E4800F041FA671CCA
:107EE000049B38B14B4A801A06FA00F018430490FC
:107EF0003C46EFE7D90644BF20228DF853201A07ED
:107F000044BF2B228DF8532022782A2A03D0079AC7
:107F100000210A200BE0039A111D12680391002A28
:107F200010DA524243F00200079204900BE0274619
:107F300001343B78303B092B03D800FB023201218E
:107F4000F5E701B107923B782E2B1ED17B782A2BC7
:107F50000AD1039B1A1D1B680392002BB8BF4FF078
:107F6000FF330237059310E000230593781C194670
:107F70000A24074601303A78303A092A03D804FB2C
:107F800001210123F5E703B1059103223978224845
:107F900000F0E6F940B14023CBEB000003FA00F01B
:107FA000049B18430490013739781C488DF8281039
:107FB00006227E1C00F0D4F988B1194B33B9039B1B
:107FC000073323F007030833039314E003AB009354
:107FD0002A46144B04A94046AFF3008007E003ABE8
:107FE00000932A460F4B04A9404600F093F8B0F1E5
:107FF000FF3F824603D0099B5344099342E7AB8974
:108000005B0601D4099801E04FF0FF301DB0BDE8D8
:10801000F08F00BFA0B10008A6B10008AAB1000807
:10802000000000008D7D00082DE9F04791461F46B5
:108030000A698B68DDF820809342B8BF1346C9F8FF
:10804000003091F8432006460C4612B10133C9F8BE
:1080500000302368990642BFD9F800300233C9F8CE
:108060000030256815F0060510D104F1190A07E063
:108070000123524639463046C04701301AD00135F7
:10808000E368D9F800209B1A9D42F1DB94F8433055
:108090002268003318BF012392060FD5E1185A1C3D
:1080A000302081F84300224494F8451082F84310B0
:1080B000023303E04FF0FF30BDE8F08704F14302E4
:1080C00039463046C0470130F4D02268D9F8005014
:1080D000E36802F00602042A08BF5D1B2269A36858
:1080E0000CBF25EAE57500259342C4BF9B1AED1825
:1080F0004FF000091A344D4509D001232246394674
:108100003046C0470130D5D009F10109F3E700201E
:10811000BDE8F0872DE9F04317460A7E85B06E2A48
:10812000984606460C460C9B01F1430E00F0AE80CB
:1081300011D8632A22D009D8002A00F0BB80582A1F
:1081400040F0CA8081F84520834955E0642A1ED05A
:10815000692A1CD0C0E0732A00F0B08009D86F2AC9
:108160002ED0702A40F0B8800A6842F020020A60DF
:108170003EE0752A24D0782A3AD0ADE01A6801F1A1
:108180004205111D1960136884F84230A8E0216887
:108190001A6811F0800F02D0111D196008E011F06B
:1081A000400F02F10401196002D0B2F9003000E082
:1081B0001368002B3CDA2D225B4284F8432037E021
:1081C00021681A6811F0800F02D0111D196007E0B4
:1081D00011F0400F02F10401196001D0138800E092
:1081E0001368227E5C496F2A14BF0A2208221BE012
:1081F00078225A4984F845202268186812F0800FC6
:1082000000F104051D6003D1550601D5038800E087
:108210000368D00744BF42F0200222601BB92268E5
:1082200022F0200222601022002084F8430001E0A6
:1082300049490A226568A560002D08DB206820F006
:10824000040020602BB9002D7DD175460CE0002B79
:1082500079D07546B3FBF2F002FB1033CB5C05F826
:10826000013D03460028F5D1082A0BD12368DA071F
:1082700008D5236962689A42DEBF302305F8013CC5
:1082800005F1FF35C5EB0E0323612EE008681A687F
:10829000496910F0800F03D0101D1860136808E0C2
:1082A00010F0400F02F104001860136801D019802B
:1082B00000E0196000232361754616E01A68111D5D
:1082C0001960156862680021284600F049F808B175
:1082D000401B6060636804E004F1420584F84220BA
:1082E00001232361002384F84330CDF800803B460E
:1082F00003AA21463046FFF797FE013002D14FF026
:10830000FF3026E023692A4639463046C04701300F
:10831000F5D023689B0710D5002504F1190907E063
:1083200001234A4639463046C0470130E7D001357F
:10833000E368039A9B1A9D42F2DBE068039B984234
:10834000B8BF184605E00B7884F8423004F14205C6
:108350008AE705B0BDE8F083B1B10008C2B10008FA
:1083600001F0FF01102A2BDB10F0070F08D010F8E6
:10837000013B013A8B422DD010F0070F42B3F6D1EA
:10838000F0B441EA012141EA014122F007047FF003
:1083900000070023F0E80256083C85EA010586EA5A
:1083A000010685FA47F5A3FA87F586FA47F6A5FA96
:1083B00087F68EB9EED1F0BC01F0FF0102F00702A2
:1083C00032B110F8013B013A83EA010313B1F8D14D
:1083D0000020704701387047002D06BF354603382E
:1083E000073815F0010F07D1013015F4807F02BF67
:1083F000013015F4C03F0130F0BC0138704700BFB8
:1084000010B5431E0A44914204D011F8014B03F801
:10841000014FF8E710BD884210B501EB020301D807
:10842000421E0BE09842FBD28118D21AD34204D0EC
:1084300013F8014D01F8014DF8E710BD994204D041
:1084400011F8014B02F8014FF8E710BDF8B50746E7
:1084500015460E4621B91146BDE8F840FFF7B4BBFA
:108460001AB9FFF745FC2846F8BD00F015F885421B
:108470000ED929463846FFF7A7FB044650B13146CE
:108480002A46FFF7BDFF31463846FFF731FC01E0D1
:108490003046F8BD2046F8BD51F8040C0028BEBF98
:1084A000091851F8043CC018043870474FF0FF31E8
:1084B00000F000B8062930B50CBF044D044D182457
:1084C00020462946ABBE0446204630BD23000200AC
:1084D00026000200F8B500BFF8BC08BC9E467047F5
:1084E000F8B500BFF8BC08BC9E46704717B7D1B9B5
:1084F000F7CC1238D28D303B87C3D23B16BEBE3B81
:10850000FDBCA9BB2E1FC9BC838814BD307F85BCB0
:10851000228A493D573F163EB493713EDF518B3E50
:10852000B493713E573F163E228A493D307F85BC49
:10853000838814BD2E1FC9BCFDBCA9BB16BEBE3BA3
:1085400087C3D23BD28D303BF7CC123817B7D1B9A5
:1085500030629F37A48CB8379C53C936A48C38B886
:1085600045F215B9C1559EB906B90BBA03275BBAD6
:1085700033349EBA2B84D5BA471E08BBB3D224BB72
:1085800042403EBB6E5251BB58595BBB5A2B5ABB43
:1085900023684CBB074232BB027E0DBB71E7C2BAF7
:1085A000910B4EBACDAC25B918B490395985CD3957
:1085B000D6E59438910B4EBA4CFF12BB3B6D8DBB88
:1085C0007D21E4BB6B0D25BCD4D25CBCDAC78ABC70
:1085D0000B46A5BC494DBBBC8429CABC3D48CFBC99
:1085E000BA68C8BC2BDFB3BC62BA90BCCADF3DBC62
:1085F0002E767BBB3868AF3BC710803C118ED93CD0
:10860000CC091A3DAD89453D83FC6C3DF31E873D89
:10861000E5B8933D1C959B3D4E419E3D1C959B3D71
:10862000E5B8933DF31E873D83FC6C3DAD89453D28
:10863000CC091A3D118ED93CC710803C3868AF3B3D
:108640002E767BBBCADF3DBC62BA90BC2BDFB3BCCD
:10865000BA68C8BC3D48CFBC8429CABC494DBBBC24
:108660000B46A5BCDAC78ABCD4D25CBC6B0D25BC5A
:108670007D21E4BB3B6D8DBB4CFF12BB910B4EBA11
:10868000D6E594385985CD3918B49039CDAC25B993
:10869000910B4EBA71E7C2BA027E0DBB074232BBE4
:1086A00023684CBB5A2B5ABB58595BBB6E5251BB0B
:1086B00042403EBBB3D224BB471E08BB2B84D5BA75
:1086C00033349EBA03275BBA06B90BBAC1559EB9BB
:1086D00045F215B9A48C38B89C53C936A48CB83768
:1086E00030629F376B80523AAA9935BBAD6B343BF1
:1086F000560DC23B0457F9BC2635943DFA08FCBD23
:10870000D047293E6074513FD047293EFA08FCBD4E
:108710002635943D0457F9BC560DC23BAD6B343B36
:10872000AA9935BB6B80523A5776413A71E401BB46
:108730004206F2BB5B23823C635FB23C403388BDA0
:10874000861F1CBD62F69A3EF0A20B3F62F69A3E6F
:10875000861F1CBD403388BD635FB23C5B23823CF7
:108760004206F2BB71E401BB5776413A202020203B
:1087700020202020535045435452554D2053434F01
:1087800050452020202020202000000030202020E4
:10879000202020316B2020202020202020336B201F
:1087A00020202020202020356B2020202020202069
:1087B000376B00005330000053310000533300008A
:1087C0005335000053370000533900003E000000CD
:1087D000444E5200464C540053435000464E430012
:1087E000206F6666200000002053504543000000C3
:1087F000206F66660000000020202020526164691E
:108800006F445350202020002020202020617564D8
:10881000696F2070726F636573736F720000000080
:10882000202020202020202020696B3879667700C6
:108830002020202020202020574154455246414CE2
:108840004C2053434F504520202020202000000082
:1088500030202020302E356B202020316B2020202E
:10886000312E356B202020326B202020322E356BAC
:10887000202020336B200000202564200000000011
:10888000204E3100204E3200205749442000000085
:10889000204D454420000000204E415220000000A1
:1088A000205746414C00000020202020202020207E
:1088B00020202020202020002043572000000000FE
:1088C00000000000000000000000000000000000A8
:1088D0000000000000100010001000100010001038
:1088E0000000001000000000002800280028000000
:1088F0000000000000000000000000000024002430
:10890000007C00240048007C004800480000000073
:10891000003800540050003800140054005400384F
:1089200000100000002000540058003000280054BF
:1089300000140008000000000010002800280010AB
:10894000003400480048003400000000001000100F
:108950000010000000000000000000000000000007
:10896000000800100020002000200020002000202F
:10897000001000080020001000080008000800088F
:108980000008000800100020001000380010002827
:1089900000000000000000000000000000000000D7
:1089A00000100010007C001000100000000000000B
:1089B00000000000000000000000000000000010A7
:1089C000001000100000000000000000000000384F
:1089D0000000000000000000000000000000000097
:1089E0000000000000000010000000000008000867
:1089F00000100010001000100020002000000000F7
:108A0000003800440044005400440044004400384E
:108A10000000000000100030005000100010001096
:108A20000010001000000000003800440044000462
:108A3000000800100020007C000000000038004406
:108A40000004001800040004004400380000000086
:108A500000080018002800280048007C00080008D2
:108A600000000000007C004000400078000400048A
:108A70000044003800000000003800440040007846
:108A8000004400440044003800000000007C000462
:108A9000000800100010002000200020000000004E
:108AA00000380044004400380044004400440038CA
:108AB000000000000038004400440044003C000472
:108AC000004400380000000000000000001000001A
:108AD0000000000000000010000000000000000086
:108AE0000000001000000000000000100010001046
:108AF00000000000000C003000400030000C0000BE
:108B000000000000000000000000007C0000007C6D
:108B100000000000000000000000000000600018DD
:108B2000000400180060000000000000003800444D
:108B300000040008001000100000001000000000F9
:108B400000380044004C0054005C004000400038F5
:108B50000000000000100028002800280028007CE9
:108B60000044004400000000007800440044007805
:108B70000044004400440078000000000038004435
:108B80000040004000400040004400380000000069
:108B90000070004800440044004400440048007055
:108BA00000000000007C00400040007C00400040CD
:108BB0000040007C00000000007C00400040007885
:108BC0000040004000400040000000000038004429
:108BD00000400040005C00440044003800000000F9
:108BE000004400440044007C00440044004400442D
:108BF00000000000003800100010001000100010ED
:108C0000001000380000000000040004000400040C
:108C10000004000400440038000000000044004844
:108C20000050006000500048004800440000000070
:108C30000040004000400040004000400040007CF8
:108C4000000000000044006C006C0054004400442C
:108C5000004400440000000000440064006400542C
:108C60000054004C004C0044000000000038004458
:108C70000044004400440044004400380000000068
:108C80000078004400440044007800400040004068
:108C90000000000000380044004400440044004448
:108CA00000540038000400000078004400440044F0
:108CB00000780048004800440000000000380044EC
:108CC00000400030000800040044003800000000AC
:108CD000007C0010001000100010001000100010A8
:108CE00000000000004400440044004400440044EC
:108CF0000044003800000000004400440044002804
:108D0000002800280010001000000000004400446B
:108D1000005400540054006C00280028000000009B
:108D200000440028002800100010002800280044FB
:108D3000000000000044004400280028001000103B
:108D40000010001000000000007C0004000800106B
:108D5000001000200040007C0000000000180010FF
:108D6000001000100010001000100010001000187B
:108D70000020002000100010001000100008000863
:108D80000000000000300010001000100010001063
:108D900000100010001000300010002800280044CF
:108DA00000000000000000000000000000000000C3
:108DB000000000000000000000000000000000FEB5
:108DC0000020001000000000000000000000000073
:108DD000000000000000000000380044003C004497
:108DE000004C0034000000000040004000580064C7
:108DF000004400440064005800000000000000002F
:108E000000380044004000400044003800000000EA
:108E1000000400040034004C00440044004C0034C2
:108E2000000000000000000000380044007C00400A
:108E30000044003800000000000C0010007C00100E
:108E400000100010001000100000000000000000E2
:108E50000034004C00440044004C0034000400780E
:108E600000400040005800640044004400440044B6
:108E70000000000000100000007000100010001042
:108E80000010001000000000001000000070001032
:108E90000010001000100010001000E00040004022
:108EA00000480050006000500048004400000000EE
:108EB00000700010001000100010001000100010D2
:108EC000000000000000000000780054005400542E
:108ED000005400540000000000000000005800642E
:108EE0000044004400440044000000000000000072
:108EF00000380044004400440044003800000000F2
:108F00000000000000580064004400440064005861
:108F100000400040000000000034004C00440044C9
:108F2000004C0034000400040000000000580064FD
:108F30000040004000400040000000000000000031
:108F400000380044003000080044003800000000F1
:108F500000200020007800200020002000200018C1
:108F600000000000000000000044004400440044F1
:108F7000004C0034000000000000000000440044E9
:108F80000028002800280010000000000000000059
:108F9000005400540054006C002800280000000019
:108FA00000000000004400280010001000280044C9
:108FB00000000000000000000044004400280028D9
:108FC000001000100010006000000000007C00088D
:108FD000001000200040007C00000000001800107D
:108FE00000100010002000200010001000100018D9
:108FF00000100010001000100010001000100010F1
:1090000000100010003000100010001000080008D0
:10901000001000100010003000000000000000747C
:10902000004C0000000000000000000000000000F4
:109030000000000000000000000000000000000030
:109040000000000000000000000000000000000020
:109050000000000C000C000C000C000C000C000CBC
:10906000000C000C000C000C0000000C000C0000B8
:10907000000000000000001B001B001B001B001B69
:1090800000000000000000000000000000000000E0
:109090000000000000000000000080198019801905
:1090A0008019C07FC07F80190033C07FC07F00332C
:1090B0000033003300330000000000000000001EF9
:1090C000003F807580650074003C001E000780052D
:1090D000806580658075003F001E0004000400006C
:1090E0000000007000D840D8C0D880D900730006B6
:1090F000000C801BC036C066C046C006800300005E
:10910000000000000000001E003F00330033003369
:10911000001E000CC03CC066806380618063C03E5E
:10912000801C0000000000000000000C000C000C7F
:10913000000C000C00000000000000000000000017
:10914000000000000000000000000000800000019E
:109150000003000600060004000C000C000C000CCC
:10916000000C000C00040006000600030001800053
:10917000002000100018000C000C0004000600067F
:1091800000060006000600060004000C000C001893
:10919000001000200000000C002D003F001E0033D6
:1091A00000000000000000000000000000000000BF
:1091B0000000000000000000000000000000000CA3
:1091C000000C000C000CC0FFC0FF000C000C000CD9
:1091D000000C000000000000000000000000000083
:1091E000000000000000000000000000000000007F
:1091F000000000000000000C000C00040004000847
:10920000000000000000000000000000000000005E
:109210000000001E001E0000000000000000000012
:10922000000000000000000000000000000000003E
:109230000000000000000000000000000000000C22
:10924000000C000000000000000000030003000309
:109250000006000600060006000C000C000C000CC6
:109260000018001800180000000000000000001E98
:10927000003F0033806180618061806D806D80611E
:10928000806180610033003F001E0000000000008C
:1092900000000006000E001E003600260006000634
:1092A0000006000600060006000600060006000094
:1092B000000000000000001E003F8073806180619C
:1092C000800100030006000C001800300060807F61
:1092D000807F0000000000000000001C003E0063D2
:1092E00000630003000E000E000380018001806116
:1092F0008073003F001E0000000000000000000618
:10930000000E000E001E001E00160036003600661D
:10931000807F807F0006000600060000000000003D
:109320000000007F007F006000600060006E007F32
:1093300080638001800180618073003F001E000017
:10934000000000000000001E003F803380610060CC
:10935000006E007F80738061806180618033003F98
:10936000001E0000000000000000807F807F800160
:109370000003000300060006000C000C000C0008AF
:109380000018001800180000000000000000001E77
:10939000003F8063806180610021001E003F80618A
:1093A000806180618061003F001E000000000000BD
:1093B0000000001E003F0073806180618061807347
:1093C000803F801D800180610073003F001E00000F
:1093D0000000000000000000000000000000000C81
:1093E000000C000000000000000000000000000C65
:1093F000000C000000000000000000000000000061
:1094000000000000000C000C000000000000000044
:109410000000000C000C0004000400080000000024
:109420000000000080008003000E0038006000385B
:10943000000E80038000000000000000000000001B
:1094400000000000000000000000807F807F00001E
:109450000000807F807F000000000000000000000E
:10946000000000000000000000000000004000704C
:10947000001C000780010007001C00700040000075
:1094800000000000000000000000001F803FC071CD
:10949000C060C000C00180030007000E000C000C7B
:1094A0000000000C000C0000000000000000001E86
:1094B000003F803180718063806F806D806D806F30
:1094C000806700600032003E001C000000000000C9
:1094D0000000000E000E001B001B001B001B803153
:1094E0008031803F803F8031C060C060C06000003C
:1094F000000000000000007C007E00630063006349
:109500000063007E007E0063806180618063007F75
:10951000007E0000000000000000001E003F8031BF
:109520008061006000600060006000600060806139
:109530008031003F001E0000000000000000007CA1
:10954000007F0063806380618061806180618061F1
:10955000806100630063007E007C0000000000006A
:109560000000807F807F0060006000600060007FFE
:10957000007F0060006000600060807F807F0000EE
:10958000000000000000807F807F006000600060BD
:109590000060007F007F006000600060006000608D
:1095A00000600000000000000000001E003F80314D
:1095B0008061006000600060806380638061806122
:1095C0008031803F001E000000000000000080612C
:1095D00080618061806180618061807F807F806147
:1095E0008061806180618061806100000000000016
:1095F0000000003F003F000C000C000C000C000CB1
:10960000000C000C000C000C000C003F003F0000A0
:1096100000000000000080018001800180018001C5
:109620008001800180018001806180618073003F42
:10963000001E0000000000000000C06080610063A8
:1096400000660066006C0078007C006600660063BF
:1096500080618061C06000000000000000000060C8
:1096600000600060006000600060006000600060FA
:10967000006000600060807F807F000000000000CC
:109680000000C071C071C07BC07AC06AC06AC06E81
:10969000C064C060C060C060C060C060C0600000E6
:1096A00000000000000080718071807980798079ED
:1096B000806D806D806D8065806780678067806366
:1096C00080630000000000000000001E003F003327
:1096D0008061806180618061806180618061806182
:1096E0000033003F001E0000000000000000007E6C
:1096F000007F80638061806180618063007F007E85
:109700000060006000600060006000000000000079
:109710000000001E003F0033806180618061806135
:1097200080618061806580670033803F401E00005B
:10973000000000000000007E007F80638061806187
:109740008063007F007E006600630063806180614B
:10975000C0600000000000000000000E001F80310B
:10976000803100300038001E000780038061806176
:109770008031003F001E0000000000000000C0FF1C
:10978000C0FF000C000C000C000C000C000C000CC6
:10979000000C000C000C000C000C0000000000008D
:1097A0000000806180618061806180618061806192
:1097B00080618061806180618073003F001E0000D5
:1097C000000000000000C060C060C06080318031D7
:1097D0008031001B001B001B001B000E000E000E42
:1097E00000040000000000000000C0C0C0C0C0C0F5
:1097F000C0C0C0C0C0CC804C804C805E80528052C3
:109800008073806180610000000000000000C0C023
:10981000806080610033003B001E000C000C001EC5
:10982000001F003B80718061C0C00000000000008C
:109830000000C0C08061806100330033001E001E44
:10984000000C000C000C000C000C000C000C0000C4
:10985000000000000000803F803F80010003000303
:109860000006000C000C0018001800300060807F1B
:10987000807F000000000000000F000F000C000CB3
:10988000000C000C000C000C000C000C000C000C78
:10989000000C000C000C000C000F000F0000001862
:1098A00000180018000C000C000C000C000600064C
:1098B0000006000600030003000300000000000093
:1098C000001E001E00060006000600060006000638
:1098D0000006000600060006000600060006000658
:1098E000001E001E0000000C000C001E00120033C1
:1098F0000033806180610000000000000000000073
:109900000000000000000000000000000000000057
:109910000000000000000000000000000000000047
:109920000000000000000000E0FF00000000003820
:109930000018000C00000000000000000000000003
:109940000000000000000000000000000000000017
:1099500000000000000000000000001F803F806148
:109960008001801F803F80618063807FC03800005D
:109970000000000000000060006000600060006EF9
:10998000007F807380618061806180618073007F6F
:10999000006E000000000000000000000000000059
:1099A0000000001E003F80738061006000608061E5
:1099B0008073003F001E00000000000000008001D6
:1099C000800180018001801D803F80738061806103
:1099D000806180618073803F801D00000000000076
:1099E00000000000000000000000001E003F0073A7
:1099F0008061807F807F00608071003F001E0000DA
:109A0000000000000000C007C00F000C000C807FA9
:109A1000807F000C000C000C000C000C000C000CF3
:109A2000000C00000000000000000000000000002A
:109A3000801D803F80738061806180618061807360
:109A4000803F801D80018063007F003E0000006039
:109A5000006000600060006F807F807180618061C5
:109A60008061806180618061806100000000000091
:109A700000000006000600000000003E003E000658
:109A800000060006000600060006000600060000AC
:109A9000000000000006000600000000003E003E3E
:109AA0000006000600060006000600060006000686
:109AB00000060046007E003C000000600060006080
:109AC0000060806100630066006C007C00760063CB
:109AD00000638061C0600000000000000000003EE4
:109AE000003E00060006000600060006000600060E
:109AF0000006000600060006000600000000000048
:109B00000000000000000000000080DDC0FFC0CEAB
:109B1000C0CCC0CCC0CCC0CCC0CCC0CCC0CC000071
:109B20000000000000000000000000000000006FC6
:109B3000807F8071806180618061806180618061EF
:109B40008061000000000000000000000000000034
:109B50000000001E003F8073806180618061806131
:109B60008073003F001E00000000000000000000A5
:109B700000000000006E007F807380618061806162
:109B800080618073007F006E006000600060006094
:109B90000000000000000000801D803F8073806195
:109BA0008061806180618073803F801D80018001C1
:109BB000800180010000000000000000000000673C
:109BC000803F00390030003000300030003000307D
:109BD0000030000000000000000000000000000055
:109BE0000000001E803F80610060007F803F800198
:109BF0008061007F001E00000000000000000000E7
:109C0000000800180018007F007F001800180018D6
:109C1000001800180018801F800F000000000000CE
:109C20000000000000000000000080618061806191
:109C300080618061806180618063807F803D000001
:109C40000000000000000000000000000000C060F4
:109C5000803180318031001B001B001B000E000E84
:109C600000060000000000000000000000000000EE
:109C7000000080DD80DD80DD005500550055007757
:109C80000077002200220000000000000000000019
:109C9000000000000000806100330033001E000C53
:109CA000000C001E00330033806100000000000043
:109CB00000000000000000008061806180310033FE
:109CC0000033001B001B001B000E000E000E001CCA
:109CD000007C007000000000000000000000C07F59
:109CE000C07F800100030006000C00180030C07F18
:109CF000C07F00000000000080038007000600060F
:109D0000000600060006000E001C001C000E0006E7
:109D10000006000600060006800780030006000615
:109D20000006000600060006000600060006000603
:109D300000060006000600060006000600060006F3
:109D40000038003C000C000C000C000C000C000E55
:109D500000070007000E000C000C000C000C000CAB
:109D6000003C00380000000000000000000000007F
:109D700000008038807F00470000000000000000E5
:109D800000000000000000006937AC316821223378
:109D9000B40F14336821A2333863ED3EDA0F493F24
:109DA0005E987B3FDA0FC93F00010000B89D0008B4
:109DB000BCAD0008B80100000000803F00000000BA
:109DC00043EC7F3FB00AC93C0FB17F3F2FFB483DBA
:109DD0006D4E7F3F05A9963D6DC47E3F36BDC83DA3
:109DE00024137E3F73B2FA3DAC3A7D3F8340163E6A
:109DF000283B7C3FA2102F3EBE147B3FC2C5473E8E
:109E00009DC7793F135C603EF853783FCCCF783ED6
:109E100007BA763F938E883E0BFA743F31A0943E8A
:109E20004714733FE59AA03E0809713FD47CAC3ECD
:109E30009ED86E3F2A44B83E5E836C3F15EFC33E0A
:109E4000A7096A3FCA7BCF3ED86B673F80E8DA3EFE
:109E500059AA643F7533E63E98C5613FEA5AF13E20
:109E600005BE5E3F275DFC3E1A945B3F3D9C033F71
:109E70005348583F9BF5083F31DB543FDA390E3FDA
:109E80003D4D513F2A68133F029F4D3FC07F183F11
:109E900012D1493FD17F1D3F03E4453F9967223FDF
:109EA00070D8413F5636273FF9AE3D3F4AEB2B3F36
:109EB0004268393FBB85303FF304353FF304353FFB
:109EC000BB85303F4268393F4AEB2B3FF9AE3D3FFF
:109ED0005636273F70D8413F9967223F03E4453FFC
:109EE000D17F1D3F12D1493FC07F183F029F4D3F98
:109EF0002A68133F3D4D513FDA390E3F31DB543F65
:109F00009BF5083F5348583F3D9C033F1A945B3FE5
:109F1000275DFC3E05BE5E3FEA5AF13E98C5613FB3
:109F20007533E63E59AA643F80E8DA3ED86B673F56
:109F3000CA7BCF3EA7096A3F15EFC33E5E836C3FE5
:109F40002A44B83E9ED86E3FD47CAC3E0809713F8F
:109F5000E59AA03E4714733F31A0943E0BFA743F3C
:109F6000938E883E07BA763FCCCF783EF853783F41
:109F7000135C603E9DC7793FC2C5473EBE147B3F20
:109F8000A2102F3E283B7C3F8340163EAC3A7D3FDB
:109F900073B2FA3D24137E3F36BDC83D6DC47E3F8B
:109FA00005A9963D6D4E7F3F2FFB483D0FB17F3F8A
:109FB000B00AC93C43EC7F3F000000000000803F36
:109FC000B00AC9BC43EC7F3F2FFB48BD0FB17F3FB8
:109FD00005A996BD6D4E7F3F36BDC8BD6DC47E3FA1
:109FE00073B2FABD24137E3F834016BEAC3A7D3F68
:109FF000A2102FBE283B7C3FC2C547BEBE147B3F8C
:10A00000135C60BE9DC7793FCCCF78BEF853783FD4
:10A01000938E88BE07BA763F31A094BE0BFA743F88
:10A02000E59AA0BE4714733FD47CACBE0809713FCB
:10A030002A44B8BE9ED86E3F15EFC3BE5E836C3F08
:10A04000CA7BCFBEA7096A3F80E8DABED86B673FFC
:10A050007533E6BE59AA643FEA5AF1BE98C5613F1E
:10A06000275DFCBE05BE5E3F3D9C03BF1A945B3F6F
:10A070009BF508BF5348583FDA390EBF31DB543FD8
:10A080002A6813BF3D4D513FC07F18BF029F4D3F0F
:10A09000D17F1DBF12D1493F996722BF03E4453FDD
:10A0A000563627BF70D8413F4AEB2BBFF9AE3D3F34
:10A0B000BB8530BF4268393FF30435BFF304353FF9
:10A0C000426839BFBB85303FF9AE3DBF4AEB2B3FFD
:10A0D00070D841BF5636273F03E445BF9967223FFA
:10A0E00012D149BFD17F1D3F029F4DBFC07F183F96
:10A0F0003D4D51BF2A68133F31DB54BFDA390E3F63
:10A10000534858BF9BF5083F1A945BBF3D9C033FE3
:10A1100005BE5EBF275DFC3E98C561BFEA5AF13EB1
:10A1200059AA64BF7533E63ED86B67BF80E8DA3E54
:10A13000A7096ABFCA7BCF3E5E836CBF15EFC33EE3
:10A140009ED86EBF2A44B83E080971BFD47CAC3E8D
:10A15000471473BFE59AA03E0BFA74BF31A0943E3A
:10A1600007BA76BF938E883EF85378BFCCCF783E3F
:10A170009DC779BF135C603EBE147BBFC2C5473E1E
:10A18000283B7CBFA2102F3EAC3A7DBF8340163ED9
:10A1900024137EBF73B2FA3D6DC47EBF36BDC83D89
:10A1A0006D4E7FBF05A9963D0FB17FBF2FFB483D88
:10A1B00043EC7FBFB00AC93C000080BF0000000034
:10A1C00043EC7FBFB00AC9BC0FB17FBF2FFB48BDB6
:10A1D0006D4E7FBF05A996BD6DC47EBF36BDC8BD9F
:10A1E00024137EBF73B2FABDAC3A7DBF834016BE66
:10A1F000283B7CBFA2102FBEBE147BBFC2C547BE8A
:10A200009DC779BF135C60BEF85378BFCCCF78BED2
:10A2100007BA76BF938E88BE0BFA74BF31A094BE86
:10A22000471473BFE59AA0BE080971BFD47CACBEC9
:10A230009ED86EBF2A44B8BE5E836CBF15EFC3BE06
:10A24000A7096ABFCA7BCFBED86B67BF80E8DABEFA
:10A2500059AA64BF7533E6BE98C561BFEA5AF1BE1C
:10A2600005BE5EBF275DFCBE1A945BBF3D9C03BF6D
:10A27000534858BF9BF508BF31DB54BFDA390EBFD6
:10A280003D4D51BF2A6813BF029F4DBFC07F18BF0D
:10A2900012D149BFD17F1DBF03E445BF996722BFDB
:10A2A00070D841BF563627BFF9AE3DBF4AEB2BBF32
:10A2B000426839BFBB8530BFF30435BFF30435BFF7
:10A2C000BB8530BF426839BF4AEB2BBFF9AE3DBFFB
:10A2D000563627BF70D841BF996722BF03E445BFF8
:10A2E000D17F1DBF12D149BFC07F18BF029F4DBF94
:10A2F0002A6813BF3D4D51BFDA390EBF31DB54BF61
:10A300009BF508BF534858BF3D9C03BF1A945BBFE1
:10A31000275DFCBE05BE5EBFEA5AF1BE98C561BFAF
:10A320007533E6BE59AA64BF80E8DABED86B67BF52
:10A33000CA7BCFBEA7096ABF15EFC3BE5E836CBFE1
:10A340002A44B8BE9ED86EBFD47CACBE080971BF8B
:10A35000E59AA0BE471473BF31A094BE0BFA74BF38
:10A36000938E88BE07BA76BFCCCF78BEF85378BF3D
:10A37000135C60BE9DC779BFC2C547BEBE147BBF1C
:10A38000A2102FBE283B7CBF834016BEAC3A7DBFD7
:10A3900073B2FABD24137EBF36BDC8BD6DC47EBF87
:10A3A00005A996BD6D4E7FBF2FFB48BD0FB17FBF86
:10A3B000B00AC9BC43EC7FBF00000080000080BF32
:10A3C000B00AC93C43EC7FBF2FFB483D0FB17FBFB4
:10A3D00005A9963D6D4E7FBF36BDC83D6DC47EBF9D
:10A3E00073B2FA3D24137EBF8340163EAC3A7DBF64
:10A3F000A2102F3E283B7CBFC2C5473EBE147BBF88
:10A40000135C603E9DC779BFCCCF783EF85378BFD0
:10A41000938E883E07BA76BF31A0943E0BFA74BF84
:10A42000E59AA03E471473BFD47CAC3E080971BFC7
:10A430002A44B83E9ED86EBF15EFC33E5E836CBF04
:10A44000CA7BCF3EA7096ABF80E8DA3ED86B67BFF8
:10A450007533E63E59AA64BFEA5AF13E98C561BF1A
:10A46000275DFC3E05BE5EBF3D9C033F1A945BBF6B
:10A470009BF5083F534858BFDA390E3F31DB54BFD4
:10A480002A68133F3D4D51BFC07F183F029F4DBF0B
:10A49000D17F1D3F12D149BF9967223F03E445BFD9
:10A4A0005636273F70D841BF4AEB2B3FF9AE3DBF30
:10A4B000BB85303F426839BFF304353FF30435BFF5
:10A4C0004268393FBB8530BFF9AE3D3F4AEB2BBFF9
:10A4D00070D8413F563627BF03E4453F996722BFF6
:10A4E00012D1493FD17F1DBF029F4D3FC07F18BF92
:10A4F0003D4D513F2A6813BF31DB543FDA390EBF5F
:10A500005348583F9BF508BF1A945B3F3D9C03BFDF
:10A5100005BE5E3F275DFCBE98C5613FEA5AF1BEAD
:10A5200059AA643F7533E6BED86B673F80E8DABE50
:10A53000A7096A3FCA7BCFBE5E836C3F15EFC3BEDF
:10A540009ED86E3F2A44B8BE0809713FD47CACBE89
:10A550004714733FE59AA0BE0BFA743F31A094BE36
:10A5600007BA763F938E88BEF853783FCCCF78BE3B
:10A570009DC7793F135C60BEBE147B3FC2C547BE1A
:10A58000283B7C3FA2102FBEAC3A7D3F834016BED5
:10A5900024137E3F73B2FABD6DC47E3F36BDC8BD85
:10A5A0006D4E7F3F05A996BD0FB17F3F2FFB48BD84
:10A5B00043EC7F3FB00AC9BC00000000920E493C4A
:10A5C000B10AC93C2BC3163D2EFB483D752B7B3D84
:10A5D00004A9963D80B6AF3D36BDC83D2FBCE13DD8
:10A5E00073B2FA3D87CF093E8340163EB5AB223E9B
:10A5F000A2102F3ECF6E3B3EC2C5473E0115543ED2
:10A60000135C603E7F9A6C3ECCCF783EC07D823E2C
:10A61000938E883E229A8E3E32A0943E86A09A3E29
:10A62000E59AA03E128FA63ED47CAC3EEF63B23ECC
:10A630002A44B83E491DBE3E15EFC33E53B9C93E3C
:10A64000CA7BCF3E4136D53E80E8DA3E4F92E03EAF
:10A650007533E63EBBCBEB3EEA5AF13ECBE0F63E2D
:10A66000275DFC3EE4E7003F3D9C033F824B063FF5
:10A670009BF5083F6B9A0B3FDA390E3FCDD3103F65
:10A680002A68133FD9F6153FC07F183FC6021B3F0B
:10A69000D17F1D3FCBF61F3F9967223F25D2243F34
:10A6A0005636273F1594293F4AEB2B3FDE3B2E3F82
:10A6B000BB85303FC9C8323FF304353F233A373FAB
:10A6C0004268393F3B8F3B3FF9AE3D3F67C73F3F55
:10A6D00070D8413F01E2433F03E4453F65DE473F19
:10A6E00012D1493FF8BB4B3F029F4D3F207A4F3F6D
:10A6F0003D4D513F4918533F31DB543FE595563F9F
:10A700005348583F6AF2593F1A945B3F532D5D3FBF
:10A7100005BE5E3F2146603F97C5613F5A3C633F9F
:10A7200059AA643F880F663FD86B673F3CBF683FBC
:10A73000A7096A3F0C4B6B3F5E836C3F93B26D3F42
:10A740009ED86E3F73F56F3F0809713F5213723FF9
:10A750004714733FDD0B743F0BFA743FC6DE753F41
:10A7600007BA763FC58B773FF853783F9812793F09
:10A770009DC7793F02737A3FBE147B3FCDAC7B3FD0
:10A78000283B7C3FC9BF7C3FAC3A7D3FCCAB7D3F93
:10A7900023137E3FB0707E3F6DC47E3F580E7F3FD7
:10A7A0006D4E7F3FAB847F3F0FB17F3F97D37F3F9D
:10A7B00043EC7F3F11FB7F3F0000803F11FB7F3F59
:10A7C00043EC7F3F97D37F3F0FB17F3FAB847F3F09
:10A7D0006D4E7F3F580E7F3F6DC47E3FB0707E3F11
:10A7E00023137E3FCCAB7D3FAC3A7D3FC9BF7C3F5E
:10A7F000283B7C3FCDAC7B3FBE147B3F02737A3F4E
:10A800009DC7793F9812793FF853783FC58B773FC2
:10A8100007BA763FC6DE753F0BFA743FDD0B743F17
:10A820004714733F5213723F0809713F73F56F3F2E
:10A830009ED86E3F93B26D3F5E836C3F0C4B6B3F77
:10A84000A7096A3F3CBF683FD86B673F880F663FE8
:10A8500059AA643F5A3C633F97C5613F2146603F18
:10A8600005BE5E3F532D5D3F1A945B3F6AF2593F30
:10A870005348583FE595563F31DB543F4918533F05
:10A880003D4D513F207A4F3F029F4D3FF8BB4B3F1C
:10A8900012D1493F65DE473F03E4453F01E2433FB4
:10A8A00070D8413F67C73F3FF9AE3D3F3B8F3B3FCD
:10A8B0004268393F233A373FF304353FC9C8323F36
:10A8C000BB85303FDE3B2E3F4AEB2B3F1594293FA3
:10A8D0005636273F25D2243F9967223FCBF61F3FAC
:10A8E000D17F1D3FC6021B3FC07F183FD9F6153FE1
:10A8F0002A68133FCDD3103FDA390E3F6B9A0B3FD6
:10A900009BF5083F824B063F3D9C033FE4E7003F39
:10A91000275DFC3ECBE0F63EEA5AF13EBBCBEB3E78
:10A920007533E63E4F92E03E80E8DA3E4136D53E52
:10A93000CA7BCF3E53B9C93E15EFC33E491DBE3E4B
:10A940002A44B83EEF63B23ED47CAC3E128FA63EA2
:10A95000E59AA03E86A09A3E32A0943E229A8E3E70
:10A96000938E883EC07D823ECCCF783E7F9A6C3EEF
:10A97000135C603E0115543EC2C5473ECF6E3B3E60
:10A98000A2102F3EB5AB223E8340163E87CF093E34
:10A9900073B2FA3D2FBCE13D36BDC83D80B6AF3D38
:10A9A00004A9963D752B7B3D2EFB483D2BC3163DE0
:10A9B000B10AC93C920E493C00000000920E49BC0D
:10A9C000B10AC9BC2BC316BD2EFB48BD752B7BBD80
:10A9D00004A996BD80B6AFBD36BDC8BD2FBCE1BDD4
:10A9E00073B2FABD87CF09BE834016BEB5AB22BE97
:10A9F000A2102FBECF6E3BBEC2C547BE011554BECE
:10AA0000135C60BE7F9A6CBECCCF78BEC07D82BE28
:10AA1000938E88BE229A8EBE32A094BE86A09ABE25
:10AA2000E59AA0BE128FA6BED47CACBEEF63B2BEC8
:10AA30002A44B8BE491DBEBE15EFC3BE53B9C9BE38
:10AA4000CA7BCFBE4136D5BE80E8DABE4F92E0BEAB
:10AA50007533E6BEBBCBEBBEEA5AF1BECBE0F6BE29
:10AA6000275DFCBEE4E700BF3D9C03BF824B06BFF1
:10AA70009BF508BF6B9A0BBFDA390EBFCDD310BF61
:10AA80002A6813BFD9F615BFC07F18BFC6021BBF07
:10AA9000D17F1DBFCBF61FBF996722BF25D224BF30
:10AAA000563627BF159429BF4AEB2BBFDE3B2EBF7E
:10AAB000BB8530BFC9C832BFF30435BF233A37BFA7
:10AAC000426839BF3B8F3BBFF9AE3DBF67C73FBF51
:10AAD00070D841BF01E243BF03E445BF65DE47BF15
:10AAE00012D149BFF8BB4BBF029F4DBF207A4FBF69
:10AAF0003D4D51BF491853BF31DB54BFE59556BF9B
:10AB0000534858BF6AF259BF1A945BBF532D5DBFBB
:10AB100005BE5EBF214660BF97C561BF5A3C63BF9B
:10AB200059AA64BF880F66BFD86B67BF3CBF68BFB8
:10AB3000A7096ABF0C4B6BBF5E836CBF93B26DBF3E
:10AB40009ED86EBF73F56FBF080971BF521372BFF5
:10AB5000471473BFDD0B74BF0BFA74BFC6DE75BF3D
:10AB600007BA76BFC58B77BFF85378BF981279BF05
:10AB70009DC779BF02737ABFBE147BBFCDAC7BBFCC
:10AB8000283B7CBFC9BF7CBFAC3A7DBFCCAB7DBF8F
:10AB900023137EBFB0707EBF6DC47EBF580E7FBFD3
:10ABA0006D4E7FBFAB847FBF0FB17FBF97D37FBF99
:10ABB00043EC7FBF11FB7FBF000080BF11FB7FBF55
:10ABC00043EC7FBF97D37FBF0FB17FBFAB847FBF05
:10ABD0006D4E7FBF580E7FBF6DC47EBFB0707EBF0D
:10ABE00023137EBFCCAB7DBFAC3A7DBFC9BF7CBF5A
:10ABF000283B7CBFCDAC7BBFBE147BBF02737ABF4A
:10AC00009DC779BF981279BFF85378BFC58B77BFBE
:10AC100007BA76BFC6DE75BF0BFA74BFDD0B74BF13
:10AC2000471473BF521372BF080971BF73F56FBF2A
:10AC30009ED86EBF93B26DBF5E836CBF0C4B6BBF73
:10AC4000A7096ABF3CBF68BFD86B67BF880F66BFE4
:10AC500059AA64BF5A3C63BF97C561BF214660BF14
:10AC600005BE5EBF532D5DBF1A945BBF6AF259BF2C
:10AC7000534858BFE59556BF31DB54BF491853BF01
:10AC80003D4D51BF207A4FBF029F4DBFF8BB4BBF18
:10AC900012D149BF65DE47BF03E445BF01E243BFB0
:10ACA00070D841BF67C73FBFF9AE3DBF3B8F3BBFC9
:10ACB000426839BF233A37BFF30435BFC9C832BF32
:10ACC000BB8530BFDE3B2EBF4AEB2BBF159429BF9F
:10ACD000563627BF25D224BF996722BFCBF61FBFA8
:10ACE000D17F1DBFC6021BBFC07F18BFD9F615BFDD
:10ACF0002A6813BFCDD310BFDA390EBF6B9A0BBFD2
:10AD00009BF508BF824B06BF3D9C03BFE4E700BF35
:10AD1000275DFCBECBE0F6BEEA5AF1BEBBCBEBBE74
:10AD20007533E6BE4F92E0BE80E8DABE4136D5BE4E
:10AD3000CA7BCFBE53B9C9BE15EFC3BE491DBEBE47
:10AD40002A44B8BEEF63B2BED47CACBE128FA6BE9E
:10AD5000E59AA0BE86A09ABE32A094BE229A8EBE6C
:10AD6000938E88BEC07D82BECCCF78BE7F9A6CBEEB
:10AD7000135C60BE011554BEC2C547BECF6E3BBE5C
:10AD8000A2102FBEB5AB22BE834016BE87CF09BE30
:10AD900073B2FABD2FBCE1BD36BDC8BD80B6AFBD34
:10ADA00004A996BD752B7BBD2EFB48BD2BC316BDDC
:10ADB000B10AC9BC920E49BC000000800800000224
:10ADC0001000000418000006200040002800400287
:10ADD00030004004380040064000800048008002F7
:10ADE00050008004580080066000C0006800C00267
:10ADF0007000C0047800C0068000000188000003D5
:10AE00009000000598000007A0004001A800400342
:10AE1000B0004005B8004007C0008001C8008003B2
:10AE2000D0008005D8008007E000C001E800C00322
:10AE3000F000C005F800C007000100020801080288
:10AE400010010804180108062001800228014802A8
:10AE500030014804380148064001000348018802D7
:10AE60005001880458018806600180036801C80207
:10AE70007001C8047801C80680010802880108032F
:10AE80009001080598010807A0018802A80148035D
:10AE9000B0014805B8014807C0010803C80188038C
:10AEA000D0018805D8018807E0018803E801C803BC
:10AEB000F001C805F801C8070802100200020004EA
:10AEC000100210041802100620028004280250020A
:10AED0003002500438025006400200054802900239
:10AEE0005002900458029006600280056802D00269
:10AEF0007002D0047802D006800208048802100391
:10AF00009002100598021007A0028804A8025003BE
:10AF1000B0025005B8025007C0020805C8029003ED
:10AF2000D0029005D8029007E0028805E802D0031D
:10AF3000F002D005F802D00700030006080310064F
:10AF4000100318041803180620038006280390062F
:10AF5000300358043803580640030007480310071D
:10AF6000500398045803980660038007680390070D
:10AF70007003D8047803D8068003080688031806EF
:10AF80009003180598031807A0038806A8039806DD
:10AF9000B0035805B8035807C0030807C8031807CB
:10AFA000D0039805D8039807E0038807E8039807BB
:10AFB000F003D805F803D80708048004100420041F
:10AFC0001804200628048005300460043804600654
:10AFD00040040006480488045004A0045804A00655
:10AFE00060041006680488057004E0047804E00634
:10AFF000880480069004200598042007A004080611
:10B00000A8048007B0046005B8046007C0042006E7
:10B01000C8048806D004A005D804A007E0041806D8
:10B02000E8048807F004E005F804E00708052005B7
:10B0300010058005180528062805900530058805A7
:10B0400038056806400500074805200750058007B9
:10B050005805A80660050807680598057005880763
:10B060007805E8068805900698052807A0052806B3
:10B07000A8059007B0052807B8056807C0051007A0
:10B08000C8059806D0059007D805A807E005180759
:10B09000E8059807F0059807F805E8071806300650
:10B0A0003806700640060007480680075006080765
:10B0B0005806B00660061007680690077006180765
:10B0C0007806F0068806A00698063007A806A007AE
:10B0D000B0068807B8067007C0062007C806A00794
:10B0E000D0062807D806B007E0063007E806A8070C
:10B0F000F0069807F806F007480750073807980742
:10B1000050076007580770076007C0076807D00737
:10B110007807F0077007E007B807F007A807B0073F
:10B12000D807F007C807E007E807F00773717274E3
:10B13000660000003A747400000000000000000087
:10B1400000000000000000000000000000000000FF
:10B1500000000000000000000000000000000000EF
:10B1600000000000000000000000000000000000DF
:10B1700000000000000000000000000000000000CF
:10B1800000000000000000000000000000000000BF
:10B1900000000000000000004300000098010020B3
:10B1A000232D302B2000686C4C00656667454647B0
:10B1B0000030313233343536373839414243444533
:10B1C00046003031323334353637383961626364A2
:08B1D0006566000000000000AC
:08B1D8000C50FF7F0100000094
:10B1E000000000000000000000000000000000005F
:10B1F000000000000000000000000000000000004F
:10B20000000000000000000000000000000000003E
:10B21000000000000000000000000000000000002E
:10B22000000000000000000000000000000000001E
:10B23000000000000000000000000000000000000E
:10B2400000000000000000000000000000000000FE
:10B2500000000000000000000000000000000000EE
:10B2600000000000000000000000000000000000DE
:10B2700000000000000000000000000000000000CE
:10B2800000000000000000000000000000000000BE
:10B2900000000000000000000000000000000000AE
:10B2A000000000000000000000000000000000009E
:10B2B000000000000000000000000000000000008E
:10B2C000000000000000000000000000000000007E
:10B2D000000000000000000000000000000000006E
:10B2E000000000000000000000000000000000005E
:10B2F000C80000000100000001040000020000007E
:10B30000232354454D4E41494F474B4457525553C3
:10B310002323515A594358424A50234C23465648F6
:10B32000303923382323233723232323232F2D3678
:10B33000312323232323232332232323332334358D
:10B34000000101000F0000006400000096000000F2
:10B350000300000001000000960000002000000033
:10B36000070A0000C08800080B1200002C9000089B
:10B3700001000000ADDEFECA0000000038B1000888
:10B3800058B1000878B1000800000000000000007B
:10B39000000000000000000098B10008000000005C
:10B3A000000000000000000000000000000000009D
:10B3B000000000000000000000000000000000008D
:10B3C000000000000000000000000000000000007D
:10B3D000000000000000000098010020AD010008FE
:04B3E00089010008D7
:0400000508000000EF
:00000001FF
